:100000000C94B1040C94C3040C94C3040C94B9284C
:100010000C94A0310C94C3040C94C3040C94C3043A
:100020000C94C3040C94C3040C94C3040C94FC15EA
:100030000C94C3040C94C3040C94C3040C94C30424
:100040000C9415180C94C3040C9490130C94521334
:100050000C94C3040C94C3040C94C3040C94C30404
:100060000C94C3040C94C3042B0BE312E312350B62
:10007000420B4F0B5C0BE312600BE3126E0BE312AF
:10008000780B820BB30BE312E312E3128C0B990B88
:10009000A60BD111E2110112E211051218120B1276
:1000A0001112D121D721DA21DD21E221EA21F42127
:1000B000962296229622FC21FF21082211229622C6
:1000C00096229622962296229622192223222F22C7
:1000D00037223A2243224C22522296225B225E226F
:1000E00066227022782296229622962296229622C4
:1000F000962282228822C12CC42CC92CCC2CCF2C35
:10010000D22CD52CD82CDB2CDE2CE12CED2CED2C9C
:10011000ED2CED2CED2CED2CED2CED2CE72CE42C26
:10012000EA2C342D372D3A2D3D2D402D432D462DD3
:10013000492D084AD73B3BCE016E84BCBFFDC12F81
:100140003D6C74319ABD56833DDA3D00C77F11BEC8
:10015000D9E4BB4C3E916BAAAABE000000803F05CB
:10016000A84CCDB2D44EB93836A9020C50B99186FC
:1001700088083CA6AAAA2ABE000000803F003E0DC7
:100180000A002C4C696D3A002C52583A002C4275EA
:10019000663A002C002C57506F733A002C002C4DFF
:1001A000506F733A003C446F6F72003C4368656364
:1001B0006B003C416C61726D003C486F6D65003CAA
:1001C000486F6C64003C52756E003C49646C65007D
:1001D0005D0D0A005B302E396A5F70756E63685F73
:1001E00076322E32303135313032333A000D0A005A
:1001F0003D00244E005D0D0A0020460020540020E2
:100200004D3800204D3900204D3500204D34002060
:100210004D3300204D3200204D3100204D30002064
:10022000473934002047393300204739310020470F
:10023000393000204732300020473231002047312A
:100240003900204731380020473137002047004728
:1002500033382E00473830004733004732004731EB
:10026000004730005B005D0D0A005B544C4F3A00C4
:100270005D0D0A002C005B4739323A005D0D0A0023
:100280002C003A003330003238005B47005D0D0A25
:10029000003A002C005B5052423A00290D0A00201F
:1002A0006D61782074726176656C2C206D6D002014
:1002B000616363656C2C206D6D2F7365635E320026
:1002C000206D617820726174652C206D6D2F6D69D1
:1002D0006E002C20737465702F6D6D007A007900AC
:1002E00078002028003D002400202870756E636887
:1002F00020646563617920666F7220706572696F32
:1003000064290D0A00202870756E63682073746577
:10031000707065722064656C617920696E206D690A
:1003200063726F73290D0A2434313D0020287075E3
:100330006E63682073656E736F7220757020696ECE
:10034000766572742C20626F6F6C290D0A2434302C
:100350003D00202870756E63682073656E736F7240
:1003600020646F776E20696E766572742C20626FE0
:100370006F6C290D0A2433333D00202870756E639D
:1003800068206163747561746F7220757020696E86
:10039000766572742C20626F6F6C290D0A243332DB
:1003A0003D00202870756E63682061637475617408
:1003B0006F7220646F776E20696E766572742C2080
:1003C000626F6F6C290D0A2433313D00202870754F
:1003D0006E6368206D6F6465290D0A2433303D001B
:1003E0002028686F6D696E672070756C6C2D6F6664
:1003F000662C206D6D290D0A2432393D00202868B5
:100400006F6D696E67206465626F756E63652C2021
:100410006D736563290D0A2432373D002028686F0B
:100420006D696E67207365656B2C206D6D2F6D692E
:100430006E290D0A2432363D002028686F6D696EE2
:100440006720666565642C206D6D2F6D696E290DC2
:100450000A2432353D00290D0A2432343D0020287B
:10046000686F6D696E672064697220696E76657267
:1004700074206D61736B3A002028686F6D696E6738
:10048000206379636C652C20626F6F6C290D0A24E0
:1004900032333D00202868617264206C696D697494
:1004A000732C20626F6F6C290D0A2432323D0020BC
:1004B00028736F6674206C696D6974732C20626F89
:1004C0006F6C290D0A2432313D0020287265706F4F
:1004D000727420696E636865732C20626F6F6C297B
:1004E0000D0A2432303D00202861726320746F6C45
:1004F0006572616E63652C206D6D290D0A243133A0
:100500003D0020286A756E6374696F6E206465769D
:10051000696174696F6E2C206D6D290D0A2431326A
:100520003D00290D0A2431313D0020287374617487
:100530007573207265706F7274206D61736B3A0011
:10054000202870726F62652070696E20696E766512
:1005500072742C20626F6F6C290D0A2431303D00BB
:1005600020286C696D69742070696E7320696E76DD
:100570006572742C20626F6F6C290D0A24363D0061
:1005800020287374657020656E61626C6520696EE9
:10059000766572742C20626F6F6C290D0A24353DCC
:1005A00000290D0A24343D00202864697220706FF0
:1005B000727420696E76657274206D61736B3A0097
:1005C000290D0A24333D0020287374657020706F54
:1005D000727420696E76657274206D61736B3A0077
:1005E0002028737465702069646C652064656C6193
:1005F000792C206D736563290D0A24323D00202873
:10060000737465702070756C73652C2075736563E9
:10061000290D0A24313D0024303D00242420287671
:10062000696577204772626C2073657474696E67C0
:1006300073290D0A242320287669657720232070EA
:100640006172616D6574657273290D0A24472028F3
:100650007669657720706172736572207374617456
:1006600065290D0A24492028766965772062756915
:100670006C6420696E666F290D0A244E2028766905
:100680006577207374617274757020626C6F636B30
:1006900073290D0A24783D76616C75652028736195
:1006A0007665204772626C2073657474696E672981
:1006B0000D0A244E783D6C696E652028736176655D
:1006C000207374617274757020626C6F636B290D96
:1006D0000A24432028636865636B2067636F646541
:1006E000206D6F6465290D0A245820286B696C6C95
:1006F00020616C61726D206C6F636B290D0A244858
:10070000202872756E20686F6D696E67206379634B
:100710006C65290D0A7E20286379636C65207374EB
:10072000617274290D0A2120286665656420686F4E
:100730006C64290D0A3F202863757272656E7420FF
:10074000737461747573290D0A6374726C2D78204B
:10075000287265736574204772626C290D0A000D5A
:100760000A4772626C20302E396A5F70756E63685A
:100770005F7632205B27242720666F722068656CC5
:10078000705D0D0A005D0D0A00526573746F726929
:100790006E672064656661756C74730050676D20C8
:1007A000456E6400436865636B20446F6F7200445C
:1007B000697361626C656400456E61626C656400BA
:1007C00043617574696F6E3A20556E6C6F636B652B
:1007D0006400272448277C2724582720746F20751D
:1007E0006E6C6F636B00526573657420746F206369
:1007F0006F6E74696E7565005B000D0A00486F6D61
:10080000696E67206661696C0050726F6265206670
:1008100061696C0041626F727420647572696E6701
:10082000206379636C6500536F6674206C696D6931
:10083000740048617264206C696D697400414C41B8
:10084000524D3A20000D0A00496E76616C696420B1
:1008500067636F64652049443A00556E6465666954
:100860006E65642066656564207261746500556E0E
:10087000737570706F7274656420636F6D6D616EF7
:1008800064004D6F64616C2067726F7570207669CB
:100890006F6C6174696F6E004C696E65206F766570
:1008A00072666C6F7700486F6D696E67206E6F744B
:1008B00020656E61626C656400416C61726D206CD4
:1008C0006F636B004E6F742069646C650045455022
:1008D000524F4D2072656164206661696C2E20550F
:1008E00073696E672064656661756C747300566128
:1008F0006C7565203C203320757365630053657407
:1009000074696E672064697361626C656400566126
:100910006C7565203C203000496E76616C696420FE
:1009200073746174656D656E7400426164206E75E8
:100930006D62657220666F726D61740045787065D6
:100940006374656420636F6D6D616E64206C6574A3
:10095000746572006572726F723A20006F6B0D0AD7
:10096000000011241FBECFEFD8E0DEBFCDBF26E0D0
:10097000A0E0B1E001C01D92A13EB207E1F70E94E4
:10098000C5040C94AB390C9400000E9420130E9403
:10099000A2220E9493180E948F318DE1E7E2F5E0D8
:1009A000DF011D928A95E9F781E08093270578940D
:1009B0008091BE0684FF03C081E0809328050E94D9
:1009C000EE130E94E7080E940F130E94EF340E946A
:1009D00013130E9468280E94A92C0E94E8230E94F9
:1009E00067180E9438270E94F90810922705109274
:1009F000440510924605109229050E941E15DFCF6E
:100A0000EF92FF921F93CF93DF9300D000D0CDB72A
:100A1000DEB77C01122F8091BE0685FF0BC0C70197
:100A200049835A836B837C830E94812A7C816B81FA
:100A30005A81498180912805823031F149835A8356
:100A40006B837C830E94F3138091270581111CC066
:100A50000E94372449815A816B817C81882339F037
:100A60000E94151549815A816B817C81E7CF212F26
:100A7000C7010F900F900F900F90DF91CF911F91B2
:100A8000FF90EF900C943F240F900F900F900F90D9
:100A9000DF91CF911F91FF90EF9008952F923F9299
:100AA0004F925F926F927F928F929F92AF92BF927E
:100AB000CF92DF92EF92FF920F931F93CF93DF932A
:100AC000CDB7DEB7E7970FB6F894DEBF0FBECDBF48
:100AD0009C8B8B8B1B013A0109871A872B873C87DC
:100AE000AF8A2D961FAD2D972E962FAD2E97298B61
:100AF0002F963FAD2F973D8B84E0889EA001112457
:100B00005A834983AB89BC89A40FB51FB98FA88FBD
:100B1000460D571D5B8F4A8FFA0180809180A2801D
:100B2000B3802D913D914D915C91C501B4010E941E
:100B300059356C8F7D8F8E8F9F8FF4E01F9F8001C2
:100B400011242B893C89200F311F39A328A3A3012D
:100B5000400F511F5BA34AA3DA014D905D906D9049
:100B60007C90F9012081318142815381C301B2011E
:100B70000E9459356CA37DA38EA39FA3A501940168
:100B800050582D873E874F87588BD301C201B058EC
:100B90008D839E83AF83B887E981FA81E20DF31DCF
:100BA0002C8D3D8D4E8D5F8D608171818281938111
:100BB0000E9458352B013C01F101E00FF11F2CA1DF
:100BC0003DA14EA15FA160817181828193810E94CC
:100BD00058354B015C01A30192016D857E858F859F
:100BE00098890E94703869837A838B839C83A501DE
:100BF00094016D817E818F8198850E9470389B0160
:100C0000AC0169817A818B819C810E94593569830D
:100C10007A838B839C83A50194016D857E858F8566
:100C200098890E9470384B015C01A30192016D818B
:100C30007E818F8198850E9470389B01AC01C5012F
:100C4000B4010E94583529813A814B815C810E9410
:100C5000CC352B013C019D89992399F02DEB37E38D
:100C600046E055EBC301B2010E94353887FD1DC037
:100C70002BED3FE049EC50E4C301B2010E9458352E
:100C800012C02DEB37E346E055E3C301B2010E94E9
:100C90003236181654F02BED3FE049EC50E4C30116
:100CA000B2010E9459352B013C018090BA06909008
:100CB000BB06A090BC06B090BD0629853A854B8541
:100CC0005C85CA01B9010E945935A50194010E94B1
:100CD00058359B01AC01C501B4010E9470380E94D7
:100CE000FD384B015C0120E030E040E05FE3C301F0
:100CF000B2010E94703829853A854B855C850E9437
:100D000070389F77A50194010E9439360E940F37F1
:100D10000E94A6367E8B6D8BDB01AB2B09F486C15E
:100D20004B01A12CB12CBF89BB2361F0C501B401DB
:100D30000E94D2369B01AC01C701B6010E947038F7
:100D40006B017C01C501B4010E94D2364B015C01EC
:100D50009B01AC01C301B2010E94393669877A87D1
:100D60008B879C87F989E4E0FE9FC00111242B89C1
:100D70003C89280F391F3A8B298BF101E80FF91FA5
:100D8000D9012D913D914D915C916081718182815C
:100D900093810E945835A50194010E9439366CABAD
:100DA0007DAB8EAB9FAB29853A854B855C85CA01AF
:100DB000B9010E9470389B01AC0160E070E080E0F6
:100DC00090E40E9458354B015C012BEA3AEA4AE272
:100DD0005EE369857A858B859C850E9470382B013E
:100DE0003C0120E030E040E850E4C501B4010E943D
:100DF00059359B01AC01C301B2010E94703868A74C
:100E000079A78AA79BA720E030E040E05FE3C50117
:100E1000B4010E9470386CA77DA78EA79FA7198286
:100E200001E010E0ED89FE890E171F0709F4FEC0EE
:100E3000B981BC3008F04AC02CA53DA54EA55FA5E0
:100E40006D817E818F8198850E9470384B015C0195
:100E500028A539A54AA55BA56D857E858F859889CE
:100E60000E947038A50194010E945935B62EA72E14
:100E7000982E892E2CA53DA54EA55FA56D857E8556
:100E80008F8598890E9470382B013C0128A539A5CF
:100E90004AA55BA56D817E818F8198850E947038FF
:100EA0009B01AC01C301B2010E9458356D877E875A
:100EB0008F87988BE981EF5FE9838B2D9A2DA92D80
:100EC000B82D8D839E83AF83B8876EC0B80180E054
:100ED00090E00E94D23629853A854B855C850E9438
:100EE00070384B015C010E9436366D837E838F83A0
:100EF0009887C501B4010E94F3384B015C01EA8D6B
:100F0000FB8D80819181A281B3819C01AD015058FC
:100F100029833A834B835C83AAA1BBA18D919D91C8
:100F20000D90BC91A02D88AB99ABAAABBBAB2D812A
:100F30003E814F81588569817A818B819C810E9495
:100F400070382B013C01A501940168A979A98AA9EF
:100F50009BA90E9470389B01AC01C301B2010E94A1
:100F600059356D877E878F87988BA501940169819C
:100F70007A818B819C810E9470384B015C012D81AC
:100F80003E814F81588568A979A98AA99BA90E94A9
:100F900070389B01AC01C501B4010E9458356D83C6
:100FA0007E838F83988719822D853E854F8558894A
:100FB0006C8D7D8D8E8D9F8D0E945935E88DF98DBC
:100FC00060837183828393832D813E814F81588515
:100FD0006CA17DA18EA19FA10E945935A8A1B9A1A4
:100FE0006D937D938D939C9313972CA93DA94EA946
:100FF0005FA9E989FA8960817181828193810E9468
:101000005935A989BA896D937D938D939C931397D4
:101010002F89B701A6018B899C890E9400058091C8
:101020002705811121C00F5F1F4FFCCE2F89B7010B
:10103000A601C101E7960FB6F894DEBF0FBECDBF83
:10104000DF91CF911F910F91FF90EF90DF90CF90A4
:10105000BF90AF909F908F907F906F905F904F90D8
:101060003F902F900C940005E7960FB6F894DEBFE2
:101070000FBECDBFDF91CF911F910F91FF90EF90E9
:10108000DF90CF90BF90AF909F908F907F906F90A8
:101090005F904F903F902F9008958F929F92AF92C4
:1010A000BF92CF92DF92EF92FF924B015C01809151
:1010B0002805823009F447C020E030E040EA51E4DE
:1010C000C501B4010E9470380E940F370E94A636F5
:1010D0006B017C010E94A01520E030E04AE754E457
:1010E000C501B4010E9470384B015C0182E38C9D04
:1010F000B0018D9D700D112480E090E00E94D236E9
:101100009B01AC01C501B4010E9458350E940F3704
:101110000E94A636CB010E942C28C114D10499F05C
:101120000E94F31321E0C21AD10880912705811192
:101130000AC08FEF90E722E0815090402040E1F715
:1011400000C00000EACFFF90EF90DF90CF90BF90FB
:10115000AF909F908F9008950E945D2881E00E943B
:10116000ED280E94F31380912705811104C00E948D
:10117000F9080C94682808958091440584FD26C0E0
:101180009FB7F894809144058061809344059FBF88
:101190000E9410130E94141380912805982F9C70B0
:1011A00021F490912905913089F49FB7843029F476
:1011B000F89480914605806204C0F89480914605B9
:1011C0008860809346059FBF0C94D115089580E4F4
:1011D000E7E4F5E0DF011D928A95E9F76BE675E03B
:1011E00080E00E943121811103C087E00C94AB2C78
:1011F00008956AE275E08FE595E00C948C332F92A8
:101200003F924F925F926F927F928F929F92AF9296
:10121000BF92CF92DF92EF92FF920F931F93CF93E3
:10122000DF93CDB7DEB7AB970FB6F894DEBF0FBE36
:10123000CDBF98A38F8F8AE3E7E8F5E0DF011D9229
:101240008A95E9F78BE0E7E4F5E0A8E8B5E00190DE
:101250000D928A95E1F71D8E212C312CA12CB12CF9
:1012600019A2512C1E8E66246394712C58E0452ED1
:101270009924939465E0862E8D8DEF8DF8A1E80F6B
:10128000F11D0081002309F491C29FEB900F9A3168
:1012900010F00C94D5128F5F8D8FAE01475E5F4FBB
:1012A000BE01635E7F4F8F8D98A10E947A278823AD
:1012B00011F40C94D712C98CDA8CEB8CFC8CC7011E
:1012C000B6010E943E390E94A636162F70E080E0DB
:1012D00090E00E94D4369B01AC01C701B6010E9488
:1012E000583520E030E048EC52E40E9470380E940B
:1012F000D3380E94A636073421F00D3409F450C1CA
:1013000099C1183209F432C1E8F4143160F4113192
:1013100008F0D7C0143009F45AC008F48EC01A304F
:10132000D9F10C94E3121C31B9F128F4163108F408
:10133000F7C00C94E3121E3179F1163209F47DC026
:101340000C94E3121D3309F40BC1A8F4153309F40E
:1013500061C040F41B3209F4ECC0113309F4E9C058
:101360000C94E3121C3310F00C94E31216531093F8
:101370008E0589E000C11C3540F41A3508F0B0C074
:10138000103509F49BC00C94E3121C3529F01F356D
:1013900008F4BDC00C94E3126115710531F4BE8DE3
:1013A000B1110C94D912E1E0EE8F1C3199F038F4B0
:1013B000143069F01A3009F0DBC082E02CC015331C
:1013C00049F11C3559F11E3109F0D2C013C0909279
:1013D0008705CEC06115710549F06A30710511F0BD
:1013E0000C94E31224E02093870509C0F3E0F09306
:1013F000870505C06115710521F48092870580E09D
:10140000BFC06A30710511F00C94E31236E03093DE
:101410008705F5CF87E080938705AAC06115710520
:1014200049F06A30710511F00C94E31299E0909341
:101430008705E5CF40928705E2CFAE8DA1110C94D0
:10144000D912B2E0BE8F123089F028F4112359F07E
:10145000113081F08FC0163281F0103579F11330E0
:1014600009F088C007C01092880584C0EE8DE09313
:10147000880580C0109388057DC06E317105B1F07C
:1014800048F46431710511F00C94E312F4E0F09328
:10149000880512C06832710561F06233710511F080
:1014A0000C94E31237E03093880506C080928805DB
:1014B00003C026E02093880581E062C04092880541
:1014C00059C0123129F0133139F010928C0502C045
:1014D00090928C0582E04FC082E080938C054BC0D7
:1014E0006115710549F41A3519F410928B0502C083
:1014F00090928B0583E044C06A30710511F00C9422
:10150000E3121A3511F40C94E31284E039C01D354E
:1015100019F49092890502C01092890585E02BC0CC
:10152000143119F490928A0502C010928A0586E05F
:1015300022C08E8D81110C94D912113331F4109286
:101540008D0588E093E09E8F1BC06A30710511F015
:101550000C94E31290928D0588E0A3E0AE8F10C04A
:10156000672B11F00C94E3128AE00AC087E003C0F5
:1015700080E001C081E0672B19F087E10C94F6123E
:10158000F30102C0EE0FFF1F8A95E2F7CF019F0122
:101590002A213B21232B09F44AC085E10C94F61241
:1015A000672B59F7163018F4133090F01EC01E3117
:1015B000C1F030F488EF810F823030F10C94E312E7
:1015C000143611F00C94E312909292058EE027C02D
:1015D000123039F01E3129F0111120C090928F0580
:1015E0001DC082E080938F0519C0143029F015309A
:1015F00039F09092910506C082E08093910502C077
:10160000109291058CE00BC0193021F082E080939C
:10161000900502C0109290058DE001C08BE093010F
:1016200002C0220F331F8A95E2F7C901B1CFA82A61
:10163000B92A22CE802F992787FD9095A92FB92FFF
:10164000FC01E654F109E531F10508F0BCC7EC5C9A
:10165000FF4F0C948B39C0929305D0929405E09281
:101660009505F092960580E07FC0C0929705D092D4
:101670009805E0929905F0929A0539A1316039A355
:1016800081E072C0C0929B05D0929C05E0929D05BE
:10169000F0929E0589A1826089A382E065C0C09214
:1016A0009F05D092A005E092A105F092A20599A114
:1016B000946099A383E058C01093A30584E054C0BC
:1016C000C701B6010E94A1366093A4057093A505D9
:1016D0008093A6059093A70585E046C0C092A80513
:1016E000D092A905E092AA05F092AB0586E03CC035
:1016F000C092AC05D092AD05E092AE05F092AF0578
:1017000087E032C0C092B005D092B105E092B20538
:10171000F092B30588E028C0C092B505D092B60516
:10172000E092B705F092B805A52DA1605A2E8AE087
:101730001BC0C092B905D092BA05E092BB05F092E9
:10174000BC05B52DB2605B2E8BE00EC0C092BD050E
:10175000D092BE05E092BF05F092C005E52DE46091
:101760005E2E8CE001C089E08301082E02C0000FCC
:10177000111F0A94E2F7980122213321232B09F04B
:101780001AC721E633E002C0359527958A95E2F71E
:1017900020FF09C020E030E0A901C701B6010E9486
:1017A000323687FD0AC7202A312A66CD552029F016
:1017B0003E8D311102C082E08E8F25FE0EC08091D9
:1017C000A4059091A505A091A605B091A705803824
:1017D0009649A849B1050CF0F2C68091890581307F
:1017E00031F4FE8DF230A1F520FEF3C631C08091B8
:1017F000480581112DC020FE1BC080918A058130D3
:1018000039F523E333E34BEC51E460919305709198
:10181000940580919505909196050E94703860938B
:10182000930570939405809395059093960510C049
:101830008091560590915705A0915805B091590592
:101840008093930590939405A0939505B093960586
:1018500030FC10C08091520590915305A091540521
:10186000B09155058093B0059093B105A093B20552
:10187000B093B30580918705813031F426FC02C016
:101880008CE1B4C6E89426F880918C05882341F059
:10189000813061F019A682E088A791E09FA30BC078
:1018A00022E029A731E038A71FA205C0A1E0A9A71F
:1018B00018A6B2E0BFA380918A05813021F0EE8D99
:1018C000E33091F52AC035EBE32E35E0F32E00E04E
:1018D00010E0C52CD12CC601002E02C0959587952D
:1018E0000A94E2F780FF10C023E333E34BEC51E4AA
:1018F000D7016D917D918D919C910E947038F70177
:1019000060837183828393830F5F1F4FF4E0EF0E38
:10191000F11C03301105F9F6D2CF80918D0581308D
:1019200019F424E052124DC68CE0EBE6F5E0DE013E
:101930001D9601900D928A95E1F7B1FC09C0309196
:1019400087053F8F3230B9F0383009F4B0C015C187
:1019500080918E05873010F08DE148C690914D053D
:10196000981769F3BE01635F7F4F0E94312188237E
:1019700009F439C6E4CF511002C08AE137C6C1016B
:1019800080759927892B09F47BCF6091A805709108
:10199000A9058091AA059091AB050E943E390E944D
:1019A000A6366730C8F68091A305843129F08230CD
:1019B00009F009C627FC07C68FEA2822662319F01A
:1019C00061506F8F03C090918E059F8FBE016F5F36
:1019D0007F4F8F8D0E943121882309F404C64090E7
:1019E000A305609083057090840580908505909094
:1019F0008605DE0111967D0195EBC92E95E0D92E65
:101A00002FE5A22E25E0B22E00E010E0E52DF0E05B
:101A1000FEA3EDA38DA19EA1002E02C095958795F2
:101A20000A94E2F780FF33C0F4E14F1226C0D501DB
:101A300058962D913D914D915C915B976D917D9163
:101A40008D919C910E945835F6012081318142810F
:101A500053810E945835D7016D937D938D939C934C
:101A600013970230A1F4A40193010E945835F701A5
:101A700060837183828393830AC0F60180819181A0
:101A8000A281B381F70180839183A283B3830F5F27
:101A90001F4FF4E0EF0EF11C24E0C20ED11C34E025
:101AA000A30EB11C0330110509F0B4CF0FC15520AE
:101AB00009F463CF6090830570908405809085055C
:101AC0009090860505EB15E08FE5C82E85E0D82EB1
:101AD0005E018DE0A80EB11CE12CF12CA52DB0E02B
:101AE000B8A3AF8F8F8D98A10E2C02C095958795C6
:101AF0000A94E2F780FF26C0F501208131814281FE
:101B00005381D6016D917D918D919C910E945835A4
:101B1000F80120813181428153810E945835D801DA
:101B20006D937D938D939C931397B2E0EB1214C049
:101B3000A40193010E945835F80160837183828368
:101B400093830AC0F601808D918DA28DB38DF8012B
:101B500080839183A283B383FFEFEF1AFF0A0C5FA8
:101B60001F4F24E0C20ED11C34E0A30EB11C83E051
:101B7000E816F10409F0B6CFA8C09E8D933059F451
:101B8000AF8DA53009F48FC0A73009F499C0A330F8
:101B900009F09BC080C0552099F340908B05809040
:101BA000830590908405A0908505B09086050FE58B
:101BB000C02E05E0D02E05EB15E03E01BDE06B0E1A
:101BC000711CE12CF12CE52DF0E0FEA3EDA38DA11D
:101BD0009EA10E2C02C0959587950A94E2F780FD90
:101BE0000BC0F60180819181A281B381F8018083CD
:101BF0009183A283B3833EC0FF8DF730D9F14110AA
:101C000028C0D60158962D913D914D915C915B97DE
:101C1000F30160817181828193810E945935D801DD
:101C20002D913D914D915C910E945935F801608351
:101C3000718382839383F2E0EF121CC0A5019401AB
:101C40000E945935D8016D937D938D939C93139782
:101C500011C0F6012081318142815381D8016D91FB
:101C60007D918D919C910E945935F801608371831B
:101C700082839383FFEFEF1AFF0A24E0C20ED11C88
:101C80000C5F1F4F34E0630E711C83E0E816F10413
:101C900009F09DCF75CF511001C01E8EBE016F5F40
:101CA0007F4F86E007C0511001C01E8EBE016F5FDE
:101CB0007F4F87E00E943121882309F494C405C036
:101CC00080918805823008F080C41F8E10918805AD
:101CD000183041F4552009F4B2C19E8D913009F0BD
:101CE00076C489C2AE8DA23009F0A9C11123D9F002
:101CF00020E030E0A90160919305709194058091F6
:101D00009505909196050E943236882309F461C4A6
:101D1000143028F4123058F4113029F06CC2183005
:101D200008F44CC168C2511066C21E8E8BC155208A
:101D300009F423CEFFA1EF2FF0E0FEA3EDA338A519
:101D4000232F30E03BA72AA781E090E03C0108A4C4
:101D500002C0660C771C0A94E2F70FA002C0880F3D
:101D6000991F0A94E2F7682A792A852D90E0862146
:101D70009721892B09F42FC4EE0FFF1FEE0FFF1FD1
:101D8000E957FA4FADA1BEA1AA0FBB1FAA0FBB1FF7
:101D9000A15ABA4F2D913D914D915C9166A577A5C1
:101DA00080A991A90E9458356B017C01EAA5FBA589
:101DB000EE0FFF1FEE0FFF1FE957FA4FAAA5BBA5B5
:101DC000AA0FBB1FAA0FBB1FA15ABA4F2D913D915D
:101DD0004D915C9166A577A580A991A90E9458357F
:101DE0004B015C0127FE40C0E89427F82091B5051F
:101DF0003091B6054091B7055091B80560915F05E7
:101E00007091600580916105909162050E94323663
:101E100081111CC12091B9053091BA054091BB05D3
:101E20005091BC05609163057091640580916505D2
:101E3000909166050E943236811108C12091BD053E
:101E40003091BE054091BF055091C0056091670576
:101E5000709168058091690590916A050E943236FB
:101E60008111F4C081E2C2C3F9A14F2E512C64202C
:101E70007520672809F4B1C321EF222280918A05D9
:101E8000813009F456C00AA51BA5000F111F000FD1
:101E9000111F09561A4FD8012D913D914D915C911A
:101EA000C501B4010E9458352B013C01ADA0BEA074
:101EB000AA0CBB1CAA0CBB1CF501E956FA4F5F012A
:101EC0002081318142815381C701B6010E9458357A
:101ED000A30192010E9437286B017C01D8012D914A
:101EE0003D914D915C91F501608171818281938179
:101EF0000E9437284B015C016093AC057093AD05DF
:101F00008093AE059093AF059B01AC01C701B6016C
:101F10000E9458356B017C01E894F7F82AE037ED10
:101F200043EA5BE3C701B6010E94353818164CF14D
:101F300062C187E9682E85E0782E00E010E0C201DA
:101F4000002E02C0959587950A94E2F780FF10C095
:101F500023E333E34BEC51E4D3016D917D918D91FB
:101F60009C910E947038F301608371838283938314
:101F70000F5F1F4FF4E06F0E711C03301105F9F66F
:101F800082CF20E030E040E05FE3C701B6010E946D
:101F9000353818160CF466CF2FE632E143E85AE3E1
:101FA000C501B4010E9470389B01AC01C701B601A4
:101FB0000E94353818160CF455CF1DC1552009F470
:101FC000DCCC2091B5053091B6054091B705509114
:101FD000B80560915F0570916005809161059091F1
:101FE00062050E943236811106C12091B9053091F7
:101FF000BA054091BB055091BC0560916305709195
:10200000640580916505909166050E9432368111C4
:10201000F2C02091BD053091BE054091BF055091A1
:10202000C005609167057091680580916905909180
:102030006A050E943236882309F414CFDCC02E8D45
:102040002111D9C0C1018E7D9C7FD8C080918A05A5
:102050008130B1F423E333E34BEC51E46091AC0500
:102060007091AD058091AE059091AF050E947038DA
:102070006093AC057093AD058093AE059093AF056A
:102080004090AC055090AD056090AE057090AF05E6
:1020900020E030E040E850E4C301B2010E94703813
:1020A000A30192010E9470382B013C01A701960107
:1020B000C701B6010E9470389B01AC01C301B20197
:1020C0000E9458352B013C01A5019401C501B401C2
:1020D0000E9470389B01AC01C301B2010E945835C7
:1020E0002B013C0120E030E0A9010E94323687FD3F
:1020F0007CC2C301B2010E94FD382B013C01A50145
:102100009401C701B6010E9437289B01AC01C301AD
:10211000B20190580E9439362B013C01809188050C
:10212000833021F477FA709477F870948091AC053D
:102130009091AD05A091AE05B091AF0589A39AA38A
:10214000ABA3BCA320E030E0A901BC01CD010E94FB
:10215000323687FF11C077FA709477F8709489A1AE
:102160009AA1ABA1BCA1B0588093AC059093AD05EA
:10217000A093AE05B093AF050DA11EA1000F111FD6
:10218000000F111F09561A4FA3019201C501B40196
:102190000E9470389B01AC01C701B6010E945835FE
:1021A00020E030E040E05FE30E947038D8016D939A
:1021B0007D938D939C9313970AA51BA5000F111F68
:1021C000000F111F09561A4FA3019201C701B60152
:1021D0000E9470389B01AC01C501B4010E945935C1
:1021E00020E030E040E05FE30E947038F801608357
:1021F000718382839383C1018E7D907E892B09F048
:10220000EEC18091A4059091A505A091A605B0917D
:10221000A70580935B0590935C05A0935D05B09343
:102220005E05809189058093480580919305909182
:102230009405A0919505B0919605809356059093CD
:102240005705A0935805B0935905C090B005D0909C
:10225000B105E090B205F090B305A7019601609139
:1022600052057091530580915405909155050E9437
:1022700032368823C1F080915005882321F0B701C0
:10228000A6010E9412138091B0059091B105A09112
:10229000B205B091B3058093520590935305A09376
:1022A0005405B09355058091B40580935A058091EB
:1022B000910590915005981771F0409152055091F9
:1022C000530560915405709155050E941213809139
:1022D0009105809350058091900590914F05981736
:1022E00031F00E9416138091900580934F058091E4
:1022F0008705813051F46091A8057091A9058091FE
:10230000AA059091AB050E944D0880918C058093A1
:102310004B0580918A05809349053E8D3330F9F451
:1023200080918D0580934C05813089F48091BD05A5
:102330009091BE05A091BF05B091C0058093830523
:1023400090938405A0938505B093860508C01092EC
:102350008305109284051092850510928605809160
:102360008E0590914D05981759F080934D058CE09E
:10237000FE013D96ABE6B5E001900D928A95E1F73E
:1023800080918B0580934A058091870590E0FC0140
:102390003297E830F10508F04BC0E75BFF4F0C9433
:1023A0008B39BE016F5F7F4F8F8D0E94DF1F809141
:1023B0004D059F8D89133CC08CE0FE013196ABE644
:1023C000B5E01AC0AE8DAA2349F020E040E050E00D
:1023D00060E87FEB85EB95E00E94000520E040E09F
:1023E00050E060E87FEBCE0101960E9400058CE092
:1023F000FE013196AFE5B5E001900D928A95E1F7C7
:1024000017C06FE575E086E003C06FE575E087E013
:102410000E94DF1F0DC08CE0E5EBF5E0A7E7B5E01B
:10242000EBCF8CE0E7E7F5E0DF011D928A95E9F755
:102430008091880580934705883009F464C0BE8D7B
:10244000B23009F060C0813011F1D8F0823071F102
:10245000833009F04FC0C0905605D0905705E090EA
:102460005805F09059050091AC051091AD052091EB
:10247000AE053091AF051F9289A58F9398A59F93C4
:102480002BC020E040E050E060E87FEB0AC04091C4
:102490005605509157056091580570915905209146
:1024A000480585EB95E00E94000524C0C0905605C4
:1024B000D0905705E0905805F09059050091AC0573
:1024C0001091AD052091AE053091AF0581E08F935D
:1024D000E9A5EF93F8A5FF938FA0A090480547E9E1
:1024E00055E065EB75E08FE595E00E944E050F9095
:1024F0000F900F908CE0E5EBF5E0AFE5B5E00190D3
:102500000D928A95E1F78091920580935105813073
:1025100021F40E9437351092510580918F058093E8
:102520004E05882309F45DC00E94A01590914E05C8
:1025300080912805913069F48230A1F19FB7F89419
:10254000809144058860809344059FBF0E94F313E7
:1025500029C091E09093470510924B0510924A05CF
:102560001092480510924D051092500510924F059B
:102570008230A9F0BE01635F7F4F80E00E9431216D
:10258000882389F18CE0FE013D96ABE6B5E0019031
:102590000D928A95E1F70E9410130E94141387E0B0
:1025A0000E94232D10924E051CC081E01FC082E0C6
:1025B0001DC088E11BC089E119C084E017C08BE110
:1025C00015C085E213C084E111C08EE10FC08FE118
:1025D0000DC086E10BC080E209C083E207C084E23F
:1025E00005C080E003C087E001C082E2AB960FB671
:1025F000F894DEBF0FBECDBFDF91CF911F910F9139
:10260000FF90EF90DF90CF90BF90AF909F908F9012
:102610007F906F905F904F903F902F900895089516
:10262000089508950895089508950895089590913E
:10263000020180910301891708F48058891B0895CD
:10264000E0ECF0E08081826080831092C50080E140
:102650008093C400E1ECF0E0808180618083808120
:10266000886080838081806880830895E091010183
:1026700091E09E0F903409F490E0209100019213B4
:1026800005C02091440524FFF8CF0895F0E0EF53F2
:10269000FA4F8083909301018091C1008062809302
:1026A000C10008951F920F920FB60F9211248F93BD
:1026B0009F93EF93FF9380910001E82FF0E0EF5399
:1026C000FA4F90819093C6008F5F803409F480E0C8
:1026D0008093000190910101891305C08091C10090
:1026E0008F7D8093C100FF91EF919F918F910F900B
:1026F0000FBE0F901F9018959091020180910301D9
:10270000891761F0E92FF0E0EF5FF94F80819F5F5B
:10271000903809F490E09093020108958FEF0895A6
:102720001F920F920FB60F9211242F933F934F9346
:102730005F936F937F938F939F93AF93BF93EF9329
:10274000FF938091C6008F33A9F050F4883109F1CE
:10275000813211F59FB7F89480914405886015C0C7
:10276000803471F08E37C1F49FB7F894809144059E
:1027700082600BC09FB7F89480914405816005C0CA
:102780009FB7F894809144058062809344059FBF71
:1027900014C00E94BC0811C0E091030191E09E0F9B
:1027A000903809F490E020910201921731F0F0E0A6
:1027B000EF5FF94F808390930301FF91EF91BF91F9
:1027C000AF919F918F917F916F915F914F913F91C9
:1027D0002F910F900FBE0F901F90189580910301BD
:1027E000809302010895EF92FF920F931F93CF936E
:1027F000DF93D1E008E080E2F82E10E190E4E92ECA
:10280000C0914605CC2389F1D0932805C1FF02C0B1
:1028100081E00FC0C2FF02C082E00BC0C3FF02C054
:1028200083E007C0C4FF02C084E003C0C5FF03C04B
:1028300085E00E94F92CC0FD08C08FB7F8949091F4
:102840004605109246058FBF10C081E00E94232DDF
:102850009FB7F894809144058F7E809344059FBF75
:102860008091440584FFFCCFE8CFC0914405CC2380
:1028700009F4BCC0C4FF04C081E080932705CEC02A
:10288000C0FF0AC00E9490309FB7F8948091440521
:102890008E7F809344059FBF8C2F887609F43CC0BF
:1028A00080912805882349F0982F9C7769F188301A
:1028B00021F40E94B518D093290580912805811133
:1028C00003C092E090932905C6FF09C0883011F437
:1028D000E092280580912905886080932905C3FF2F
:1028E00005C08091280585FF10932805C5FF0CC001
:1028F00086E00E94232D8091290581FDC4608460BB
:1029000080932905F09228059FB7F894809144059B
:102910008779809344059FBFC1FF48C08C2F88767C
:10292000E9F580912805882331F08075B9F180910F
:10293000290581FF33C08091290582FF1CC0809149
:102940005005882371F040915205509153056091D4
:102950005405709155050E94111380EA9FE00E9472
:102960002C2880914F05882331F00E94151388EEA2
:1029700093E00E942C280E940D24892B59F080910D
:10298000290583FD07C0009328050E94D7180E94DF
:10299000B11502C010922805109229059FB7F8942E
:1029A000809144058D7F809344059FBFC2FF1EC068
:1029B00080912805807371F08091290582FF04C001
:1029C0000E9410130E941413809129058260809345
:1029D000290504C010922905109228059FB7F89484
:1029E000809144058B7F809344059FBF809128058B
:1029F0008C7711F00E94D71880912805803251F40D
:102A00008091290581FF06C00E94D931811102C041
:102A100010932805809129058111F2CEDF91CF9185
:102A20001F910F91FF90EF9008959FB7F8948091B8
:102A300044058260809344059FBF0895CF93DF9340
:102A40000E94522D80912805813021F482E00E945D
:102A5000232D2FC00E94D931882341F08091440555
:102A60008062809344050E94F31302C010922805EF
:102A700084E091E00E94DB311CC08D3079F0DD23D1
:102A800099F1893221F4D13009F04CC0D0E00E9494
:102A90007C138F3F09F448C08A3079F7EC2FF0E0BF
:102AA000EC5FFE4F10820E94F3138091270588236C
:102AB00011F0C0E0EBCF80910401811103C00E94AE
:102AC000AB2CF7CF843229F484E091E00E94FA31F4
:102AD000F6CF80912805813011F489E0F0CF84E0B1
:102AE00091E00E94FF08EBCF813288F28F3279F2B9
:102AF0008832B1F08B33B1F0CF3428F08BE00E94F4
:102B0000AB2CC0E0C4CF2C2F30E0CF5F9FE9980FF3
:102B1000F901EC5FFE4F9A3108F480528083B7CF01
:102B2000D1E0B5CFD2E0B3CF0E9415150E94F313C8
:102B300080912705882309F4AACFDF91CF910895CA
:102B40000E9415150E94F31380912705811108C07A
:102B50000E940D24892BB1F780912805883091F3CC
:102B600008958091BE0682FF02C0289A01C028986D
:102B7000809128058C70A1F0809184018093980148
:102B800080918501809397018091B106880F8450D0
:102B900081958093960180916F00826080936F0091
:102BA000089580916F008D7F80936F0080918100E8
:102BB000887F816080938100109283018091B406A8
:102BC0008F3F21F490914605992349F09091280573
:102BD000943029F090E00E942C2881E001C080E030
:102BE0009091BE0692FF02C091E08927882311F0E0
:102BF000289A0895289808951F920F920FB60F9261
:102C000011242F933F934F935F936F937F938F93F1
:102C10009F93AF93BF93CF93DF93EF93FF938091F5
:102C200083018111EFC19BB180919801807E9F71DA
:102C3000892B8BB98BB1837E90919701892B8BB9AE
:102C40008091960186BD82E085BD81E080938301FD
:102C500078948091AA019091AB01892B09F0A4C0CE
:102C60008091880190918701981709F492C0E091B2
:102C7000880186E0E89FF0011124E455FE4FF093AF
:102C8000AB01E093AA0183819481909389008093A2
:102C90008800808191819093A6018093A501A281F3
:102CA0008091A7018A1771F1A093A70181E1A89FE4
:102CB000D0011124A053BE4FB093A901A093A80145
:102CC0001D968D919D910D90BC91A02DB695A795C7
:102CD000979587958093910190939201A09393018A
:102CE000B093940180938D0190938E01A0938F01F6
:102CF000B09390018093890190938A01A0938B01F6
:102D0000B0938C01C091A801D091A9018091840158
:102D10009881892780939801258189819A81AB8147
:102D2000BC81022E04C0B695A795979587950A9405
:102D3000D2F78093990190939A01A0939B01B0934D
:102D40009C018D819E81AF81B885022E04C0B6950D
:102D5000A795979587950A94D2F780939D019093B4
:102D60009E01A0939F01B093A00189859A85AB85B0
:102D7000BC8504C0B695A795979587952A95D2F7F7
:102D80008093A1019093A201A093A301B093A40109
:102D90000BC00E94D1159FB7F894809144058460C0
:102DA000809344059FBF2EC10E94AA2C10929701C8
:102DB0008091990190919A01A0919B01B0919C0101
:102DC0004091890150918A0160918B0170918C0131
:102DD000840F951FA61FB71F8093890190938A01C6
:102DE000A0938B01B0938C01E091A801F091A9010F
:102DF0004585568567857089481759076A077B0797
:102E000068F524E02093970145855685678570898C
:102E1000841B950BA60BB70B8093890190938A01B5
:102E2000A0938B01B0938C01208180912A05909111
:102E30002B05A0912C05B0912D0525FF04C001970D
:102E4000A109B10903C00196A11DB11D80932A05F6
:102E500090932B05A0932C05B0932D0580919D0197
:102E600090919E01A0919F01B091A00140918D0190
:102E700050918E0160918F0170919001840F951F88
:102E8000A61FB71F80938D0190938E01A0938F0191
:102E9000B093900145855685678570894817590715
:102EA0006A077B0778F520919701286020939701A6
:102EB0004585568567857089841B950BA60BB70BD6
:102EC00080938D0190938E01A0938F01B093900118
:102ED000208180912E0590912F05A0913005B09111
:102EE000310526FF04C00197A109B10903C001966D
:102EF000A11DB11D80932E0590932F05A093300541
:102F0000B09331058091A1019091A201A091A301FC
:102F1000B091A4014091910150919201609193016F
:102F200070919401840F951FA61FB71F8093910184
:102F300090939201A0939301B09394014585568597
:102F400067857089481759076A077B0778F52091CC
:102F50009701206120939701458556856785708983
:102F6000841B950BA60BB70B809391019093920154
:102F7000A0939301B09394012081809132059091A8
:102F80003305A0913405B091350527FF04C00197A2
:102F9000A109B10903C00196A11DB11D809332059D
:102FA00090933305A0933405B0933505809128059F
:102FB000843039F48091430590919701892380935F
:102FC00097018091A5019091A60101979093A60188
:102FD0008093A501892B69F41092AB011092AA018C
:102FE000809188018F5F80938801863011F4109260
:102FF000880180918501909197018927809397019D
:1030000010928301FF91EF91DF91CF91BF91AF912A
:103010009F918F917F916F915F914F913F912F91F0
:103020000F900FBE0F901F9018951F920F920FB622
:103030000F9211248F939F939BB1809185018C7186
:10304000937E892B8BB915BC9F918F910F900FBEEA
:103050000F901F901895FF920F931F93CF93DF93BC
:103060001092850110928401C0E0D0E00C2F1C2F3B
:103070002091B20630E08C2F0C2E02C0359527959A
:103080000A94E2F720FF07C0F09085010E94AF226A
:103090008F29809385012091B30630E002C03595D9
:1030A00027951A95E2F720FF08C010918401802F20
:1030B0000E94B922812B809384012196C330D105CF
:1030C000A9F6DF91CF911F910F91FF9008950E9473
:1030D000D1158BE2E4E5F1E0DF011D928A95E9F775
:1030E00083E2E9E8F1E0DF011D928A95E9F71092A9
:1030F000820110928101109288011092870181E073
:1031000080938601109283010E942B188BB1837EDD
:1031100090918501892B8BB98BB18F71909184012E
:10312000892B8BB908958AB18C618AB9209A8AB1AA
:10313000806E8AB9E1E8F0E080818F7E80838081B3
:1031400088608083E0E8F0E080818C7F80838081EC
:103150008F708083EEE6F0E08081887F808314BCEE
:1031600015BC8081816080830895CF93DF93C091E7
:103170008101D09182012097B9F081E080935501BF
:1031800060916B0170916C0180916D0190916E0165
:103190009B01AC010E947038698B7A8B8B8B9C8B66
:1031A0001092820110928101DF91CF9108952F92A8
:1031B0003F924F925F926F927F928F929F92AF92C7
:1031C000BF92CF92DF92EF92FF920F931F93CF9314
:1031D000DF93CDB7DEB7E5970FB6F894DEBF0FBE2D
:1031E000CDBF80912805807709F40AC220E030E045
:1031F000A90160916B0170916C0180916D019091BA
:103200006E010E9432368111FBC103C6809181019B
:1032100090918201892B09F4FAC180918701F6E02F
:10322000F89FF0011124E455FE4FFE83ED83809159
:103230005401828320918101309182013E872D8744
:10324000D9019596BC91BCA7F901F6A1FDA7D901BA
:103250009796BC91BEA7F901F0A5FFA720915E014A
:1032600030915F0140916001509161016CA57DA595
:103270008B2F9F2F0E94583568A779A78AA79BA7F5
:1032800020E030E0A9010E94323687FF04C018A672
:1032900019A61AA61BA620917701288F30917801D4
:1032A000398F409179014A8F50917A015B8F8091DB
:1032B0006F018C8F909170019D8FA0917101AE8FE5
:1032C000B0917201BF8FE0917B01E8A3F0917C0186
:1032D000F9A320917D012AA330917E013BA3409167
:1032E00067014CA3509168015DA3809169018EA391
:1032F00090916A019FA320917301309174014091D4
:1033000075015091760128AB39AB4AAB5BAB30917C
:103310006B01398340916C01498720906D01309099
:103320006E01509166015F878CA58C8B9DA59D8B4E
:10333000AEA5AE8BBFA5BF8B3EE3C32E33ECD32E21
:103340003EE2E32E39E3F32E188A198A1A8A1B8A81
:1033500026013701EF85E111B4C3AD85BE85919695
:103360002D913D914D915C919497C701B6010E94BA
:1033700070384B015C0120E030E040E05FE30E94E8
:1033800070389B01AC0169817985C1010E94593572
:103390009B01AC01C701B6010E9470389B01AC01D2
:1033A0006C897D898E899F890E9458358B018DABF0
:1033B0009CAB288D398D4A8D5B8D0E94323687FFFC
:1033C00086C3288D398D4A8D5B8D6CA57DA58EA514
:1033D0009FA50E9458359B01AC010E9459356B0195
:1033E0007C012C8D3D8D4E8D5F8D69817985C1016C
:1033F0000E9459359B01AC01C701B6010E943936C4
:103400006B017C0128A139A14AA15BA1688D798D4E
:103410008A8D9B8D0E943236882309F455C3B1E012
:10342000BF87FC8DF9832D8D29872E8C3F8C088DCD
:10343000198D3A8D3DAB4B8D4CABA7019601688938
:1034400079898A899B890E945935688B798B8A8B07
:103450009B8BA30192010E94323687FDF2C328A5FF
:1034600039A54AA55BA5B8018DA99CA90E9435384C
:1034700018160CF4DCC389819985D10180936B0106
:1034800090936C01A0936D01B0936E01FF85F09352
:10349000660140905A0150905B0160905C01709011
:1034A0005D0198014DA95CA9C301B2010E94703869
:1034B00069837A838B839C830E941F366B017C0116
:1034C0006091560170915701809158019091590176
:1034D0000E941F364B015C01A70196010E945835DE
:1034E0000E94A63669877A878B879C87E985FA854B
:1034F000AD81BE81ED93FC93309709F4CDC320914B
:1035000062013091630140916401509165016889C5
:1035100079898A899B890E9459352B013C0129812F
:103520003A814B815C81C501B4010E9458359B01F1
:10353000AC01C301B2010E9439364B015C01298103
:103540003A814B815C81C701B6010E945835A501C3
:1035500094010E94703860936201709363018093BC
:1035600064019093650120EC31EE44E65EE4C50110
:10357000B4010E9470380E941F360E94A636603D3A
:10358000B7E07B078105910508F0ACC3ED81FE81B2
:103590001582AD81BE8114967C936E9313978091B2
:1035A0008601809387018F5F863009F4D4C38093AE
:1035B0008601209167013091680140916901509125
:1035C0006A01B8018DA99CA90E94353818160CF023
:1035D000C5C3E0918101F0918201C801ADA9BCA9E8
:1035E00085A396A3A7A3B0A789819A81AB81BC814B
:1035F0008093560190935701A0935801B0935901BD
:103600009091880180918601981300CE02C40E9497
:103610000D241C019093820180938101009709F48D
:10362000F8C38091550110912805882319F0109254
:103630005501BEC0809154018F5F853019F0809391
:10364000540102C010925401E091540121E12E9FD7
:10365000F0011124E053FE4FF0938001E0937F01CD
:10366000D1018C91808311964D915D916D917C91EA
:10367000149703E0440F551F661F771F0A95D1F773
:10368000418352836383748315964D915D916D914F
:103690007C91189783E0440F551F661F771F8A950A
:1036A000D1F7458356836783708719964D915D9155
:1036B0006D917C911C9793E0440F551F661F771FF7
:1036C0009A95D1F741875287638774871D966D91CC
:1036D0007D918D919C9150976B017C0123E0CC0CE6
:1036E000DD1CEE1CFF1C2A95D1F7C586D686E78621
:1036F000F08A0E94D23660935601709357018093EE
:10370000580190935901F10125A136A147A150A577
:103710000E9439369B01AC0160935A0170935B01A2
:1037200080935C0190935D0160E070E080EA9FE32C
:103730000E94393660935E0170935F01809360014F
:1037400090936101109262011092630110926401E2
:1037500010926501812F8077E1F060917301709183
:103760007401809175019091760160936B01709363
:103770006C0180936D0190936E019B01AC010E94DE
:103780007038D10151966D937D938D939C9354978E
:103790000FC0F10161897289838994890E94FD3883
:1037A00060936B0170936C0180936D0190936E0137
:1037B00010926701109268011092690110926A01DB
:1037C000D10191968D909D90AD90BC909497A5015C
:1037D000940160E070E080E09FE30E9439362B01A5
:1037E0003C011077F101C5A0D6A0E7A0F0A41123F9
:1037F00009F44DC0F2E0F0936601D10151962D918C
:103800003D914D915C9154972D833E834F83588712
:103810000E9470389B01AC01C701B6010E94583567
:103820002B013C0120E030E0A9010E94323687FFE5
:103830001DC0A5019401C501B4010E945935A7011D
:1038400096010E9470389B01AC016D817E818F8151
:1038500098850E9458350E94FD38609373017093DB
:1038600074018093750190937601D7CC40926701E3
:10387000509268016092690170926A01109273011E
:10388000109274011092750110927601C6CC1092BC
:103890006601C0927701D0927801E0927901F092AE
:1038A0007A010E941D244B015C01609373017093A7
:1038B000740180937501909376019B01AC010E9485
:1038C000703869837A838B839C8300918101109186
:1038D0008201D80195962D913D914D915C919897DB
:1038E00029873A874B875C8751962D913D914D9161
:1038F0005C9154972D833E834F8358879B01AC0185
:103900006D817E818F8198850E9458359B01AC0125
:10391000C301B2010E9470389B01AC0169857A85B0
:103920008B859C850E94593520E030E040E05FE3C4
:103930000E9470386B017C0120E030E0A9010E94F8
:10394000353818160CF0ACC029853A854B855C8556
:10395000C701B6010E94323687FF8EC0F801858C00
:10396000968CA78CB0A029813A814B815C81C501DE
:10397000B4010E9458359B01AC01C301B2010E9401
:10398000703860937B0170937C0180937D019093EC
:103990007E01A70196010E94323687FF3DC0C50116
:1039A000B4010E94FD3860936F01709370018093A1
:1039B000710190937201A50194016D817E818F81C7
:1039C00098850E943236811104C0F1E0F0936601BF
:1039D00024CC2D813E814F815885C501B4010E94C0
:1039E00058359B01AC01C301B2010E9470389B01A4
:1039F000AC0160917701709178018091790190918B
:103A00007A010E9458356093770170937801809312
:103A1000790190937A0101CCC0927701D09278011C
:103A2000E0927901F0927A01C0927B01D0927C0100
:103A3000E0927D01F0927E01D80191966D917D9189
:103A40008D919C9194979B01AC010E945935A701DF
:103A500096010E94703829813A814B815C810E94D5
:103A600059350E94FD3860936F0170937001809307
:103A7000710190937201D1CBB2E0B0936601809155
:103A80006B0190916C01A0916D01B0916E018093DA
:103A90006F0190937001A0937101B0937201BDCB3F
:103AA00010927701109278011092790110927A01A8
:103AB00080926F0190927001A0927101B092720198
:103AC000ACCBE13061F041C0E2E0EF87AACCA501C8
:103AD000940169817985C1010E9459357CC0A70193
:103AE00096016C8D7D8D8E8D9F8D0E9470389B010F
:103AF000AC016C897D898E899F890E9458358B0124
:103B00008DAB9CAB28A139A14AA15BA10E943236A2
:103B100087FF93CC28A139A14AA15BA16C897D893B
:103B20008E899F890E9458352C8D3D8D4E8D5F8DDD
:103B30000E9439366B017C0108A119A15AA15DAB25
:103B40008BA18CAB92E09F8778CCAD85BE8591969A
:103B50002D913D914D915C919497C701B6010E94C2
:103B600070384B015C019B01AC0169817985C10111
:103B70000E94353818169CF520E030E040E05FE305
:103B8000C501B4010E9470389B01AC01698179853F
:103B9000C1010E9458359B01AC01C701B6010E94CA
:103BA00070389B01AC016C897D898E899F890E9448
:103BB00058358B018DAB9CAB2CA13DA14EA15FA1D3
:103BC0000E94353818165CF4A50194016981798545
:103BD000C1010E945835698379871C012ECC2CA124
:103BE0003DA14EA15FA16C897D898E899F890E942C
:103BF00058359B01AC010E9459356B017C0128A905
:103C000039A94AA95BA969817985C1010E94593501
:103C10009B01AC01C701B6010E9439366B017C01E2
:103C20000CA11DA1BEA1BDABEFA1ECAB06CC2EE358
:103C300033EC4EE259E3C301B2010E9459352B0126
:103C40003C01288939894A895B89C301B2010E94F4
:103C500058356B017C012CA13DA14EA15FA1B8019B
:103C60008DA99CA90E94353818167CF08981998508
:103C7000D10180936B0190936C01A0936D01B0937F
:103C80006E013F853093660104CC0C8B1D8B4DA9D2
:103C90004E8B5CA95F8B5ECB80912805807709F401
:103CA0002ECC10926B0110926C0110926D0110924B
:103CB0006E011092620110926301109264011092E1
:103CC0006501C0925601D0925701E0925801F092DE
:103CD0005901A3019201C701B6010E943936AD8591
:103CE000BE8570C0603AFFE07F078105910510F442
:103CF000E1E009C06034FFE17F078105910510F420
:103D0000E2E001C0E3E0AD81BE811596EC93AD81A8
:103D1000BE8115962C911597022E04C09695879515
:103D2000779567950A94D2F7E985FA8502C0EE0F78
:103D3000FF1F2A95E2F7ED93FC9361157105F1E001
:103D40008F07910508F425CC2FEF3FEFED81FE8121
:103D50003483238324CC109286012BCC20E030E0E6
:103D6000A901B8018DA99CA90E94353818160CF03C
:103D700049C010926B0110926C0110926D0110926B
:103D80006E01109262011092630110926401109210
:103D90006501C0925601D0925701E0925801F0920D
:103DA0005901009181011091820120915A013091B5
:103DB0005B0140915C0150915D01C701B6010E9419
:103DC0003936D80195966D937D938D939C939897F2
:103DD000E5960FB6F894DEBF0FBECDBFDF91CF9151
:103DE0001F910F91FF90EF90DF90CF90BF90AF9019
:103DF0009F908F907F906F905F904F903F902F900B
:103E00000C94722710928201109281010E94F92372
:103E1000F7CBE5960FB6F894DEBF0FBECDBFDF91AE
:103E2000CF911F910F91FF90EF90DF90CF90BF90B7
:103E3000AF909F908F907F906F905F904F903F904A
:103E40002F900895F999FECF92BD81BD81E08FBB7F
:103E500080B50895F894F999FECF92BD81BD81E0B7
:103E60008FBB40B54627842F992787FD9095262F35
:103E700030E082239323892B39F06F3F19F060BD26
:103E800084E006C084E104C0442321F060BD84E2E4
:103E90008FBBF99A789408959F92AF92BF92CF9278
:103EA000DF92EF92FF920F931F93CF93DF938C01DA
:103EB0007A016B01C40ED51EEB01912C5C01A61A90
:103EC000B70ACE018A0D9B1DCC15DD0591F091102E
:103ED00009C0692D772767FD7095272F221F22279C
:103EE000221F01C021E06991922E960E0E942A1F86
:103EF000E8CF692DC8018E0D9F1DDF91CF911F91D5
:103F00000F91FF90EF90DF90CF90BF90AF909F9078
:103F10000C942A1F9F92AF92BF92CF92DF92EF92A2
:103F2000FF920F931F93CF93DF938B017A016C0164
:103F3000C40ED51EEC01912C5B01A81AB90AC5016B
:103F40008C0F9D1FCC15DD0591F00E94221F911052
:103F500009C0292D332727FD3095232F221F222723
:103F6000221F01C021E0922E980E8993E8CFC8014C
:103F70008E0D9F1D0E94221F21E030E0981611F047
:103F800020E030E0C901DF91CF911F910F91FF90A8
:103F9000EF90DF90CF90BF90AF909F90089521E574
:103FA000829FC001112440E550E09D5F0C944C1F9E
:103FB00040E550E0BC018EEA93E00C944C1F2DE0EC
:103FC000829FC00111244CE050E09E5F0C944C1F76
:103FD0006AE080E090E00E942A1F46E550E061E838
:103FE00076E081E090E00C944C1FEF92FF920F93EB
:103FF0001F93CF93DF93CDB7DEB72C970FB6F8940E
:10400000DEBF0FBECDBF182F80FFC7C08AE08093F0
:10401000B10689E18093B4061092B2061092B306FD
:1040200083E08093B5068AE097EDA3E2BCE380933A
:10403000B6069093B706A093B806B093B9068FE67C
:1040400092E1A3E0BBE38093BA069093BB06A093F2
:10405000BC06B093BD061092BF0680E090E0A8ECCD
:10406000B1E48093C0069093C106A093C206B093BA
:10407000C30640E050E06AEF73E44093C4065093F7
:10408000C5066093C6067093C7068AEF90E09093CA
:10409000C9068093C80680E090E0A0E8BFE3809363
:1040A000CA069093CB06A093CC06B093CD0610928F
:1040B000BE0680E090E0AAE7B3E480938106909387
:1040C0008206A0938306B09384068093850690931E
:1040D0008606A0938706B0938806809389069093FE
:1040E0008A06A0938B06B0938C0640938D0650935E
:1040F0008E0660938F0670939006409391065093BE
:10410000920660939306709394064093950650939D
:104110009606609397067093980640E050EA6CE02C
:1041200077E44093990650939A0660939B067093A8
:104130009C0640939D0650939E0660939F06709345
:10414000A0064093A1065093A2066093A306709325
:10415000A40640E050E068E473EC4093A506509359
:10416000A6066093A7067093A8064093A9065093ED
:10417000AA066093AB067093AC064093AD065093CD
:10418000AE066093AF067093B0061092CF06109201
:10419000D0061092CE060E94E81F11FF10C0CE017B
:1041A00001967C018CE0F70111928A95E9F700E015
:1041B000B701802F0E94DF1F0F5F0830C9F712FF81
:1041C0000AC060E080E093E00E942A1F60E081E581
:1041D00093E00E942A1F13FF05C060E08EEA93E07F
:1041E0000E942A1F2C960FB6F894DEBF0FBECDBFDB
:1041F000DF91CF911F910F91FF90EF9008951F9342
:10420000CF93DF93182FEB0181E5189FB0011124A4
:104210007D5F40E550E0CE010E948A1F892B39F472
:104220001882BE01812F0E94CF1F80E001C081E073
:10423000DF91CF911F910895CF93DF93EC0140E57B
:1042400050E06EEA73E00E948A1F892B31F41882D5
:10425000CE010E94D81F80E001C081E0DF91CF91A4
:1042600008951F93CF93DF93182FEB018DE0189FD4
:10427000B00111247E5F4CE050E0CE010E948A1F05
:10428000892B59F48CE0FE0111928A95E9F7BE0161
:10429000812F0E94DF1F80E001C081E0DF91CF917C
:1042A0001F91089580E090E00E94221F8A3059F407
:1042B00046E550E061E070E081E896E00E948A1FE8
:1042C00021E0892B09F420E0822F0895CF92DF921C
:1042D000EF92FF92CF93DF93C82F6A017B0120E01A
:1042E00030E0A901C701B6010E94323687FD1CC12A
:1042F000C43608F445C02CE92C0F80E02330B8F513
:1043000030E0823079F0F901EE0FFF1FEE0FFF1F52
:10431000833011F1813019F0EF57F94F23C0E35783
:10432000F94F20C0E901CC0FDD1FCC0FDD1FC756B0
:10433000D94F20E030E040E752E4C701B6010E94C7
:10434000703820E030E040E752E40E947038688323
:1043500079838A839B83E4C0EB55F94FF7FAF09495
:10436000F7F8F094C082D182E282F382D9C08F5FE5
:104370002A3008F4DBC0843009F4D8C02A50BECFFC
:10438000C701B6010E943E390E94A6368C2F90E0EC
:104390008A32910508F0CAC0FC01EF5AFF4F0C9415
:1043A0008B39633008F4C4C06093B106B9C0609320
:1043B000B406B6C06093B20602C06093B3060E9412
:1043C0002B18AEC08091BE06662311F0846007C032
:1043D0008B7F05C08091BE06662321F080648093A8
:1043E000BE069EC08F7BFBCF8091BE06662311F078
:1043F0008068F5CF8F77F3CF6093B50691C0C092F8
:10440000B606D092B706E092B806F092B90688C018
:10441000C092BA06D092BB06E092BC06F092BD06EE
:104420007FC08091BE06662311F08160D8CF8E7F59
:10443000D6CF8091BE06662321F084FF7BC08062C8
:10444000CECF8F7DCCCF8091BE06662311F08860E1
:1044500001C0877F8093BE060E94682861C080915A
:10446000BE06662311F08061BACF8F7CB8CF60930F
:10447000BF0656C0C092C006D092C106E092C206E6
:10448000F092C3064DC0C092C406D092C506E09219
:10449000C606F092C70644C070E07093C9066093E8
:1044A000C8063EC0C092CA06D092CB06E092CC06A7
:1044B000F092CD0635C06093CE0632C08091CF0613
:1044C000662311F0826009C08D7F07C08091CF06FE
:1044D000662311F0816001C08E7F8093CF0620C0DB
:1044E0008091D006662311F0826007C08D7F05C0E1
:1044F0008091D006662321F081608093D00610C0A1
:104500008E7FFBCF70E07093D2066093D10608C017
:10451000C092D306D092D406E092D506F092D60689
:104520000E94E81F80E007C084E005C083E003C06C
:1045300086E001C08AE0DF91CF91FF90EF90DF909D
:10454000CF9008950E945221811108C087E00E94F7
:10455000AB2C8FEF0E94F51F0C945A2D08958823E1
:1045600021F0813021F488E0089584E0089580E10D
:104570000895882321F0813021F480E4089580E2B9
:10458000089580E80895882321F0813021F484E0A3
:10459000089582E0089588E008954F925F926F92A7
:1045A0007F928F929F92AF92BF92CF92DF92EF92C3
:1045B000FF920F931F93CF93DF931091430211113A
:1045C00001C012E1115000914102101709F4EFC02F
:1045D00089E2189FE0011124CB5BDD4F8D889E8816
:1045E000AF88B88C69A17AA18BA19CA19B01AC0179
:1045F0000E9459352DA13EA14FA158A50E947038A7
:104600006B017C019B01AC01B401C5010E943236F3
:1046100087FF02C064017501A601B701498B5A8B5F
:104620006B8B7C8B111101C012E177247A94710E8F
:10463000701619F029E2622E27C0809144020813F7
:1046400051C00E94B5184EC0679C800111240B5BBD
:104650001D4F711002C092E1792E7A94809144022C
:10466000781202C00E94B518F801C588D688E7887C
:10467000F08CA701960161897289838994890E94CF
:104680003236811106C0E801809141027812DCCFF8
:1046900029C0F80161A172A183A194A19B01AC0181
:1046A0000E945935F80125A136A147A150A50E94C5
:1046B000703829893A894B895C890E9459354B01A8
:1046C0005C01A70196010E943236F80187FF05C000
:1046D000818A928AA38AB48AD6CFC18AD28AE38A8F
:1046E000F48AD1CF60904102F9E26F9E80011124DB
:1046F0000B5B1D4F77247394760C82E1781201C016
:10470000712C5090430289E2482E751409F44DC073
:10471000479CE0011124CB5BDD4FF8018188928832
:10472000A388B488C988DA88EB88FC88A701960139
:10473000C501B4010E94323687FF23C0F80161A190
:1047400072A183A194A19B01AC010E945935F8018B
:1047500025A136A147A150A50E9470389B01AC014C
:10476000C501B4010E9459354B015C01A7019601B6
:104770000E94323687FF05C0898A9A8AAB8ABC8A32
:10478000672C2D893E894F89588D69897A898B8953
:104790009C890E943236811101C0672C7394F2E12A
:1047A0007F1201C0712C8E01B0CF60924102DF9167
:1047B000CF911F910F91FF90EF90DF90CF90BF901E
:1047C000AF909F908F907F906F905F904F900895E3
:1047D0008CE1E5E2F2E0DF011D928A95E9F71092A3
:1047E00044021092430281E08093420210924102FF
:1047F00008959091440280914302891769F081E005
:10480000890F823109F480E020914102921302C0A5
:1048100080934102809344020895809144029091D4
:104820004302981739F029E2829FC00111248B5B63
:104830009D4F089580E090E00895E0914402EF5F7D
:10484000E23109F4E0E080914302E81761F089E287
:10485000E89FF0011124EB5BFD4F61897289838928
:1048600094890C94FD3860E070E0CB01089581E0FC
:104870002091440290914202291380E008952F92E2
:104880003F924F925F926F927F928F929F92AF92E0
:10489000BF92CF92DF92EF92FF920F931F93CF932D
:1048A000DF93CDB7DEB7AD970FB6F894DEBF0FBE7E
:1048B000CDBF142F052F6B8F7C8F822E209143024A
:1048C00039E2239F10011124F101EB5BFD4F1F0121
:1048D000158616861786108A15A216A217A210A68C
:1048E000108249E956E766E97EE741A352A363A334
:1048F00074A35C0141E8E42E46E0F42E9E01235FA0
:104900003F4F38A32F8F85E292E09E8F8D8F6F01EE
:10491000FE013196FAA3E9A3912CF5016191719101
:10492000819191915F01F701208131814281538111
:104930000E9470380E944038EF8DF8A16193719306
:1049400081939193F8A3EF8FED8DFE8D419051905F
:1049500061907190FE8FED8F641975098609970932
:104960002B013C0197FF07C0442455243201461A0D
:10497000570A680A790AF601418252826382748278
:10498000F101258536854785508942165306640610
:10499000750610F429013A01F101458656866786AD
:1049A000708A0E94D436F70120813181428153817F
:1049B0000E9439362B013C01E9A1FAA16193719360
:1049C00081939193FAA3E9A320E030E0A9010E942A
:1049D000323687FF0AC0F1019081892D9DA70E9480
:1049E000B9229DA5892BF1018083A3019201C30106
:1049F000B2010E947038F10125A136A147A150A54E
:104A00000E945935F10165A376A387A390A79394DB
:104A1000F4E0EF0EF11C24E0C20ED11C33E093123F
:104A20007CCF0E94FD386B017C01F10165A376A368
:104A300087A390A785859685A785B089892B8A2B22
:104A40008B2B09F4FCC120E030E0A901612F702F0D
:104A50008B8D9C8D0E94323687FD21C0882061F0AD
:104A6000A7019601612F702F8B8D9C8D0E9470384D
:104A7000162F072F8B8F9C8F20E030E040E85FE3FC
:104A8000612F702F8B8D9C8D0E94323687FF0DC059
:104A900010E000E030E83B8F8FE38C8F06C019E90F
:104AA00006E7F6E9FB8F2EE72C8FA701960160E061
:104AB00070E080E89FE30E94393669A77AA78BA748
:104AC0009CA7E1E3F2E0FAA3E9A32DE836E038A3DE
:104AD0002F8FCE010D969A8F898FFE013196FE8F12
:104AE000ED8FC12CD12C7601ED8DFE8D80809180D3
:104AF000A280B38020E030E0A901C501B4010E948A
:104B00003236882309F47FC029A53AA54BA55CA5B8
:104B1000C501B4010E9470384B015C01ED8DFE8D22
:104B200060837183828393839B01AC0160E070E0BA
:104B300080E89FE30E9439362B013C01E89477F826
:104B4000EF8DF8A12081318142815381C301B201EF
:104B50000E9470386BA37CA38DA39EA39B01AC0124
:104B6000612F702F8B8D9C8D0E94323687FF06C07F
:104B70001BA30CA3FB8DFDA32C8D2EA3F101F1A192
:104B8000FB8FF101F2A1FC8FF101F3A1FFA3F10171
:104B9000F4A1F8A7EF8DF8A12485358546855785C2
:104BA000C301B2010E9470383B018C019B01AC0132
:104BB0006B8D7C8D8FA198A50E94323687FF04C033
:104BC0006B8C7C8C0FA118A5C301D801F10181A3C6
:104BD00092A3A3A3B4A3E9A1FAA1208131814281C8
:104BE0005381C501B4010E9470389B01AC01C7011B
:104BF000B6010E9458356B017C011BA10CA1FDA1DF
:104C0000FB8F2EA12C8F8D8D9E8D04969E8F8D8F68
:104C1000E9A1FAA13496FAA3E9A32F8D38A12C5F5C
:104C20003F4F38A32F8FE98DFA8D8E179F0709F01C
:104C30005BCF9091430280914402981306C0F1012A
:104C4000118A128A138A148A0BC024EA30E74DE7CE
:104C50005FE3C701B6010E943538181634F4F1013C
:104C6000118E128E138E148E5BC024EA30E74DE74E
:104C70005FEBC701B6010E943538181644F034EADC
:104C8000C32E30E7D32E3DE7E32E3FEBF32EA701F3
:104C9000960160E070E080E89FE30E94583520E0D4
:104CA00030E040E05FE30E9470380E94FD386B0105
:104CB0007C012091B6063091B7064091B80650911C
:104CC000B906F10161A172A183A194A10E9470387B
:104CD000A70196010E9470384B015C01A701960163
:104CE00060E070E080E89FE30E9458359B01AC01D2
:104CF000C501B4010E9439366B017C0120E030E02F
:104D0000A9010E94323687FF04C0C12CD12CE12CAE
:104D1000F12CA601B701F101418F528F638F748F7F
:104D2000212F302F4B8D5C8D612F702F8B8D9C8DA3
:104D30000E947038162F072FF82EE92E862F902FFD
:104D4000AF2DBE2DF101858F968FA78FB0A3A18CBB
:104D5000B28CC38CD48C60903D0270903E028090E7
:104D60003F02909040029301A401612F702F8F2D7C
:104D70009E2D0E94323687FD0BC09301A401B50120
:104D8000C6010E94323687FD11C0530164010EC076
:104D9000212F302F4F2D5E2DB501C6010E943236D6
:104DA00087FD04C0A12EB02ECF2CDE2CC501D6016C
:104DB000F101858B968BA78BB08F8CE0FE0131962D
:104DC000A1E3B2E001900D928A95E1F7812F902F37
:104DD000AF2DBE2D80933D0290933E02A0933F02E3
:104DE000B09340028CE0FE013D96A5E2B2E0019056
:104DF0000D928A95E1F780914202809343028F5F82
:104E0000823109F480E080934202AD960FB6F894A7
:104E1000DEBF0FBECDBFDF91CF911F910F91FF90ED
:104E2000EF90DF90CF90BF90AF909F908F907F904A
:104E30006F905F904F903F902F900C94CD22AD9645
:104E40000FB6F894DEBF0FBECDBFDF91CF911F919B
:104E50000F91FF90EF90DF90CF90BF90AF909F9019
:104E60008F907F906F905F904F903F902F9008951C
:104E700080912A0590912B05A0912C05B0912D05CC
:104E80008093250290932602A0932702B0932802D4
:104E900080912E0590912F05A0913005B09131059C
:104EA0008093290290932A02A0932B02B0932C02A4
:104EB0008091320590913305A0913405B09135056C
:104EC00080932D0290932E02A0932F02B093300274
:104ED00008958091430290914402891708F48E5EF0
:104EE000891B08950E94B518809144028093410265
:104EF0000C94CD226F927F928F929F92AF92BF922D
:104F0000CF92DF92EF92FF920F931F93CF93DF9395
:104F10007C018B016A01FB018081F701E80FF11D23
:104F20002081EF012D3229F4229621816624639499
:104F300007C02B3211F0219602C022962181612CEC
:104F4000A12CB12C712C60E070E0CB01FE0130EDA2
:104F5000932E920E29E02915C8F0B39428E02B1562
:104F600088F0A1107A94A5E0B0E09B01AC010E940A
:104F70009139660F771F881F991F690D711D811D5B
:104F8000911D0BC0A11009C0739407C02EEF92129F
:104F900007C0A11005C0AA24A39421962081D6CFD2
:104FA000BB2009F449C00E94D2364B015C0120E0CD
:104FB00030E0A9010E943236882361F18FEF781624
:104FC0006CF42AE037ED43E25CE3C501B4010E94D2
:104FD00070384B015C0173947394F0CF78120BC05E
:104FE0002DEC3CEC4CEC5DE3C501B4010E94703843
:104FF0004B015C010FC0772069F020E030E040E217
:1050000051E4C501B4010E9470384B015C017A94EF
:1050100017149CF3662021F0B7FAB094B7F8B09457
:10502000F60180829182A282B382CE19DF09C1503B
:10503000F801C08381E001C080E0DF91CF911F9132
:105040000F91FF90EF90DF90CF90BF90AF909F9027
:105050008F907F906F900895009741F0EFE9FFE007
:105060003197F1F700C000000197F6CF08958F92B5
:105070009F92AF92BF92CF92DF92EF92FF9269011F
:105080007A019B01AC010E9470384B015C01A701C1
:105090009601C701B6010E9470389B01AC01C501A1
:1050A000B4010E945935FF90EF90DF90CF90BF90F0
:1050B000AF909F908F900C94FD38EBE6F0E08081EC
:1050C000817F8083E8E6F0E080818E7F8083089591
:1050D00084B1817F84B985B18E6085B98091BE0627
:1050E00083FF0BC080916B008E6080936B0080917A
:1050F000680081608093680008950C945D28CF92C9
:10510000DF92FF920F931F93CF93DF931F92CDB740
:10511000DEB793B19E708091BE0686FD02C08EE020
:1051200098279923D9F0C12CD12CF12C01E010E063
:105130008C2D99830E94C3229981892339F098018B
:105140000C2C01C0220F0A94EAF7F22A8FEFC81A3A
:10515000D80AE3E0CE16D10459F701C0F12C8F2D07
:105160000F90DF91CF911F910F91FF90DF90CF9023
:1051700008951F920F920FB60F9211242F933F9311
:105180004F935F936F937F938F939F93AF93BF934F
:10519000EF93FF9380912805813071F0809146054F
:1051A00081110AC00E94BC089FB7F89480914605FF
:1051B0008360809346059FBFFF91EF91BF91AF91B0
:1051C0009F918F917F916F915F914F913F912F911F
:1051D0000F900FBE0F901F9018952F923F924F92F5
:1051E0005F926F927F928F929F92AF92BF92CF9277
:1051F000DF92EF92FF920F931F93CF93DF93CDB780
:10520000DEB766970FB6F894DEBF0FBECDBF582E3F
:105210008091270581115CC185EAA82E86E0B82E11
:105220009E01235F3F4F190100E010E0C12CD12CFB
:105230007601652C712C802F0E94AF22D1018D93B5
:105240001D01C301002E02C0959587950A94E2F7CF
:1052500080FF1AC020E030E040EC5FEBF501608198
:105260007181828193810E947038688B472E4C0136
:10527000262F372FAC01C701B6010E94353818160A
:105280001CF0C888D42C74010F5F1F4FF4E0AF0EE0
:10529000B11C0330110579F68090C4069090C506C4
:1052A000A090C606B090C70624E0288B01E06AE211
:1052B00075E0CE0101960E948C332090BF06312C00
:1052C000FE0131968AE295E09E8B8D8B80E090E026
:1052D000412C10E0B701A60170589301082E02C0BE
:1052E000359527950A94E2F720FF28C04394AD89AD
:1052F000BE891D921D921D921C9213979101082E3A
:1053000002C0359527950A94E2F720FF03C00023D9
:1053100019F007C0002329F0C082D182E282F38213
:1053200004C040835183628373832DE030E02C0FEF
:105330003D1F280F391FD9012C91122B019634964D
:105340002D893E892C5F3F4F3E8B2D8B83309105FD
:1053500021F6642D70E080E090E00E94D2360E9439
:10536000FD389B01AC01C501B4010E947038AB014E
:10537000BC0110934305498B5A8B6B8B7C8B0E942D
:10538000382720E049895A896B897C89CE010196AA
:105390000E943F240E94D7180E94B1150023E9F013
:1053A0000E947F28FE013D9620E030E090E0619170
:1053B000462F412359F0AC01022E02C05595479566
:1053C0000A94E2F740FF02C0609516232F5F3F4F1B
:1053D0002330310561F7109343050E94D71880915F
:1053E00044058473C1F080914405807329F00E94C4
:1053F000BC080E94F3136CC0011165C00E947F2895
:105400008521A9F79FB7F894809144058B7F8093FD
:1054100044059FBF04C0812F8C7109F0BFCF0E944B
:1054200067180E94E8238091C8069091C9060E94DF
:105430002C2831E00327C9F020E030E040EA50E4B6
:105440006091CA067091CB068091CC069091CD06F2
:105450000E9470386B017C018090C0069090C1065C
:10546000A090C206B090C30610C0C090CA06D090EB
:10547000CB06E090CC06F090CD068090C4069090CC
:10548000C506A090C606B090C70688898150888B53
:1054900081110DCFEAE2F5E080E090E09301082E63
:1054A00002C0359527950A94E2F720FF04C01082C8
:1054B000118212821382019634968330910571F71E
:1054C0000E94382705C08091440582FF9BCF8FCF73
:1054D00066960FB6F894DEBF0FBECDBFDF91CF91B9
:1054E0001F910F91FF90EF90DF90CF90BF90AF9002
:1054F0009F908F907F906F905F904F903F902F90F4
:1055000008958F929F92AF92BF92CF92DF92EF92C7
:10551000FF920F931F93CF93DF93C090BF06D12CC0
:1055200025EAE22E26E0F22E8C01C0E0D0E0C60192
:105530000C2E02C0959587950A94E2F7F8018080B9
:105540009180A280B38020E030E0A90180FF15C0E7
:10555000C501B4010E94323687FD20C0F701808169
:105560009181A281B3819C01AD015058C501B40164
:105570000E943538181694F040C0C501B4010E944D
:10558000353818165CF0F701208131814281538152
:10559000C501B4010E94323687FF2FC080912805D3
:1055A0008830C1F00E94BC089FB7F89480914605EE
:1055B0008560809346059FBFDF91CF911F910F912A
:1055C000FF90EF90DF90CF90BF90AF909F908F9023
:1055D0000C94F3139FB7F8948091440588608093EE
:1055E00044059FBF0E94F3138091270581110FC0CE
:1055F000809128058111F6CFD5CF2196F4E0EF0EEA
:10560000F11C0C5F1F4FC330D10509F090CFDF9123
:10561000CF911F910F91FF90EF90DF90CF90BF90AF
:10562000AF909F908F900895CF93DF93EC01899175
:10563000882319F00E943613FACFDF91CF91089595
:10564000CF93DF93FC018491EF012196882321F011
:105650000E943613FE01F7CFDF91CF910895EF92AC
:10566000FF920F931F93CF93DF931F92CDB7DEB7B7
:10567000262FEDB6FEB66DB77EB7641B71090FB667
:10568000F8947EBF0FBE6DBF0DB71EB70F5F1F4FE3
:10569000302FF8019E2F931B941728F4622F0E943D
:1056A0005D399193F7CF442361F0F801E40FF11DC8
:1056B00031978081805D49830E9436134981415032
:1056C000F2CF0FB6F894FEBE0FBEEDBE0F90DF9185
:1056D000CF911F910F91FF90EF90089548E062E005
:1056E0000C942F2B8A3020F0843620F442E003C043
:1056F00041E001C043E06AE00C942F2BBF92CF92AF
:10570000DF92EF92FF920F931F93CF93DF93CDB76A
:10571000DEB72A970FB6F894DEBF0FBECDBF611576
:1057200071058105910591F480E32A960FB6F894EE
:10573000DEBF0FBECDBFDF91CF911F910F91FF90C4
:10574000EF90DF90CF90BF900C94361320E03AE0BA
:10575000C32ED12CE12CF12CBB24B394B20E01E06A
:1057600010E00C0F1D1F020F111DA70196010E94D2
:105770006939F8016083B901CA01611571058105B4
:10578000910511F02B2DE8CFBB2049F0FE01EB0D68
:10579000F11D8081805D0E943613BA94F5CF2A9660
:1057A0000FB6F894DEBF0FBECDBFDF91CF911F9132
:1057B0000F91FF90EF90DF90CF90BF9008958F9260
:1057C0009F92AF92BF92CF92DF92EF92FF920F9390
:1057D0001F93CF93DF93CDB7DEB72A970FB6F89418
:1057E000DEBF0FBECDBF6B017C01142F20E030E087
:1057F000A9010E94323687FF07C08DE20E9436134E
:10580000F7FAF094F7F8F094012F023060F020E0FE
:1058100030E048EC52E4C701B6010E9470386B01D9
:105820007C010250F2CF10FF0AC020E030E040E2DD
:1058300051E4C701B6010E9470386B017C0120E081
:1058400030E040E05FE3C701B6010E9459350E9495
:10585000A136E1E0F0E0EC0FFD1FE10FF11D2EE2BB
:105860002083D12C5AE0852E912CA12CB12C6115CE
:10587000710581059105A9F0D11201C0D394EE24E0
:10588000E394F12CEC0EFD1EED0CF11CA50194012E
:105890000E946939605DF7016083B901CA01D39440
:1058A000E6CF80E3D11648F4E1E0F0E0EC0FFD1F15
:1058B000ED0DF11D8083D394F5CF8D2DD1120BC04A
:1058C000D394D3948F5FE1E0F0E0EC0FFD1FE80F7D
:1058D000F11D80E38083DD2041F0FE01ED0DF11D1F
:1058E00080810E943613DA94F6CF2A960FB6F89488
:1058F000DEBF0FBECDBFDF91CF911F910F91FF9003
:10590000EF90DF90CF90BF90AF909F908F900895D1
:105910002091BE0620FF08C02BE832E441E25DE39F
:105920000E94703844E001C043E00C94DF2B2091CA
:10593000BE0620FF08C02BE832E441E25DE30E948E
:10594000703841E001C040E00C94DF2B43E00C9440
:10595000DF2B08950895CF93C82F811103C08CE5E4
:1059600099E044C084E599E00E94202B4C2F50E040
:10597000FA013197E631F10580F5E558FF4F0C94B7
:105980008B398CE399E002C08AE299E00E94202BD7
:105990002BC088E199E0FACF8EE099E0F7CF8DEF48
:1059A00098E0F4CF8EEE98E0F1CF8DEC98E0EECF5A
:1059B00084EC98E0EBCF89EB98E0E8CF86EA98E0BA
:1059C000E5CF88E998E0E2CF82E898E0DFCF8EE685
:1059D00098E0DCCF8AE598E0D9CF88E498E00E948F
:1059E000202B8C2F0E94722B85E498E0CF910C9491
:1059F000202BCF93C82F8DE398E00E94202BC3303B
:105A000091F03CF4C13061F0C230A1F487E298E03B
:105A10000FC0C43059F0C53069F48DEF97E008C06D
:105A200082E398E005C084E198E002C089E098E054
:105A30000E94202B8AEF97E00E94202B84EF91E0B8
:105A4000CF910C942C28CF93C82F88EF97E00E9419
:105A5000202B8C2F90E0FC013197E830F105E8F421
:105A6000EF56FF4F0C948B3986EE97E014C082ED11
:105A700097E011C080EC97E00EC088EB97E00BC078
:105A80008FEA97E008C084EA97E005C08CE997E0C8
:105A900002C089E897E00E94202B85E897E0CF912B
:105AA0000C94202B8FE597E00C94202B8BE196E053
:105AB0000C94202BFF920F931F93CF93DF9387E1DA
:105AC00096E00E94202B8091B1060E94722B8EEFEF
:105AD00095E00E94202B8091B4060E94722B80EEEC
:105AE00095E00E94202B8091B2060E94722B87ECD9
:105AF00095E00E94202B8091B2060E946E2B80ECD4
:105B000095E00E94202B8091B3060E94722B88EAB8
:105B100095E00E94202B8091B3060E946E2B81EAB3
:105B200095E00E94202B8091BE0682FB882780F999
:105B30000E94722B80E895E00E94202B8091BE0687
:105B400086FB882780F90E94722B80E695E00E94F0
:105B5000202B8091BE06881F8827881F0E94722BE9
:105B600080E495E00E94202B8091B5060E94722B64
:105B70008AE295E00E94202B8091B5060E946E2B50
:105B800082E295E00E94202B6091B6067091B706E4
:105B90008091B8069091B9060E94A62C82E095E00B
:105BA0000E94202B6091BA067091BB068091BC06C2
:105BB0009091BD060E94A62C87EE94E00E94202BB7
:105BC0008091BE0681700E94722B8AEC94E00E9444
:105BD000202B8091BE0685FB882780F90E94722BBE
:105BE0008FEA94E00E94202B8091BE0683FB8827D9
:105BF00080F90E94722B84E994E00E94202B80910E
:105C0000BE06829581700E94722B88E794E00E9404
:105C1000202B8091BF060E94722B8EE594E00E949B
:105C2000202B8091BF060E946E2B86E594E00E9497
:105C3000202B6091C0067091C1068091C2069091A0
:105C4000C3060E94A62C89E394E00E94202B609159
:105C5000C4067091C5068091C6069091C7060E9441
:105C6000A62C8CE194E00E94202B8091C8060E9413
:105C7000722B8DEF93E00E94202B6091CA067091E9
:105C8000CB068091CC069091CD060E94A62C80EE8A
:105C900093E00E94202B8091CE060E94722B8CEC08
:105CA00093E00E94202B8091CF06869581700E9400
:105CB000722B82EA93E00E94202B8091CF068170A4
:105CC0000E94722B8AE793E00E94202B8091D006DD
:105CD000869581700E94722B82E593E00E94202BB2
:105CE0008091D00681700E94722B8CE293E00E941A
:105CF000202B6091D1067091D20680E090E00E9446
:105D00007E2B85E093E00E94202B6091D30670915A
:105D1000D4068091D5069091D6060E94A62C89EED5
:105D200092E00E94202B84E6F82E10E0C1E8D6E035
:105D300000E087EE92E00E94202B802F8F0D0E94C2
:105D4000722B85EE92E00E94202B123071F01330FE
:105D5000B9F0113029F0688179818A819B8117C05F
:105D60006C857D858E859F8512C020E030E041E600
:105D700055E4688D798D8A8D9B8D0E94393607C0D8
:105D80008CA19DA1AEA1BFA1BC01CD0190580E94E4
:105D9000A62C82EE92E00E94202B013029F00230E6
:105DA00031F080EE92E005C08EED92E002C08CED05
:105DB00092E00E94202B123051F0133059F0113034
:105DC00019F082ED92E008C080EC92E005C08FEA05
:105DD00092E002C08FE992E00E94202B8BE992E0D2
:105DE0000E94202B0F5F2496033009F0A2CF8AE097
:105DF000F80E1F5F8CE8F81299CFDF91CF911F91B9
:105E00000F91FF900895CF9385E992E00E94202B97
:105E1000C0E06C2F86E395E00E9472330E94882CCC
:105E2000C23021F083E992E00E94202BCF5FC33083
:105E300081F781E992E00E94202B809142050E9427
:105E4000722B8DE892E0CF910C94202BEF92FF9271
:105E50000F931F93CF93DF93CDB7DEB72C970FB679
:105E6000F894DEBF0FBECDBFF12CBE016F5F7F4F38
:105E70008F2D0E943121811104C087E00E94AB2C3C
:105E800069C08AE892E00E94202B86E0F81631F083
:105E9000E7E0FE1208C084E892E002C087E892E0E2
:105EA0000E94202B04C086E38F0D0E94722B82E893
:105EB00092E00E94202B8E010F5F1F4FE12CF80112
:105EC00061917191819191918F010E94882CF2E0F2
:105ED000EF1619F080E892E002C08CE792E00E9491
:105EE000202BE39483E0E812EACFF394E8E0FE127B
:105EF000BCCF86E792E00E94202B07E715E0F12C4B
:105F0000F80161917191819191918F010E94882C8A
:105F1000F2E0FF1619F084E792E002C080E792E019
:105F20000E94202BF39483E0F812EACF8AE692E0F5
:105F30000E94202B609183057091840580918505D6
:105F4000909186050E94882C86E692E00E94202B84
:105F50000E94032F2C960FB6F894DEBF0FBECDBF64
:105F6000DF91CF911F910F91FF90EF90089584E6FC
:105F700092E00E94202B80914705823091F038F406
:105F8000882361F08130A9F48EE592E00CC0833063
:105F900069F0883071F484E592E005C081E692E012
:105FA00002C08BE592E00E94202B0CC088E592E0B5
:105FB000FACF8FE492E00E94202B80914705825017
:105FC0000E94722B8CE492E00E94202B80914D0560
:105FD0008A5C0E94722B80914B05813049F028F039
:105FE000823051F48DE392E005C087E492E002C074
:105FF00082E492E00E94202B80914905811103C028
:1060000088E392E002C083E392E00E94202B80911B
:106010004A05811103C08EE292E002C089E292E05B
:106020000E94202B80914805813019F484E292E08F
:1060300002C08FE192E00E94202B80914E058130BA
:1060400049F028F0823051F483E192E005C08BE101
:1060500092E002C087E192E00E94202B80915005DF
:10606000813031F040F0823051F48BE092E005C095
:106070008FE092E002C087E092E00E94202B8091A6
:106080004F05882329F0823039F48FEF91E002C068
:1060900083E092E00E94202B8CEF91E00E94202B65
:1060A00080915A050E94722B89EF91E00E94202B6B
:1060B000609156057091570580915805909159054A
:1060C0000E94972C85EF91E00C94202B1F93CF9387
:1060D000DF93182FEB0182EF91E00E94202B812F9C
:1060E0000E94722B80EF91E00E94202BCE010E9433
:1060F000142B8DEE91E0DF91CF911F910C94202B0A
:10610000CF93DF93EC0184ED91E00E94202BCE0130
:106110000E94142B80ED91E0DF91CF910C94202B05
:10612000BF92CF92DF92EF92FF920F931F93CF9384
:10613000DF93CDB7DEB768970FB6F894DEBF0FBE1A
:10614000CDBF8CE0EAE2F5E0DE011D9601900D92F4
:106150008A95E1F7809128058430E9F040F4813098
:10616000E9F080F0823009F58BEA91E01CC08031C3
:1061700079F018F4883049F018C0803291F08034FA
:1061800021F013C08AEC91E00EC085EC91E00BC0C9
:106190008FEB91E008C089EB91E005C082EB91E0C4
:1061A00002C085EA91E00E94202B8091B5068370A1
:1061B00039F0BE01635F7F4FCE0101960E948C33A0
:1061C0008091B50680FD05C08091B50681FF6DC048
:1061D0001FC08EE991E00E94202B69817A818B811A
:1061E0009C810E94882C8CE991E00E94202B6D817B
:1061F0007E818F8198850E94882C8CE991E00E9495
:10620000202B69857A858B859C850E94882CDCCF24
:1062100085E991E00E94202B9BE6E92E95E0F92E7E
:106220008E010F5F1F4FB12C6801F70161917191D1
:10623000819191917F0120853185428553850E940E
:1062400059359B01AC01F801608171818281938194
:106250000E945835F8016083718382839383F2E052
:10626000BF120FC0209183053091840540918505B0
:10627000509186050E945835F801608371838283AE
:1062800093830C5F1F4FF60160817181828193813E
:106290000E94882CF2E0BF1621F083E991E00E9471
:1062A000202BB39423E0B212BFCF8091B50682FFBA
:1062B00008C08DE891E00E94202B0E9469270E946F
:1062C000722B8091B50683FF08C088E891E00E9498
:1062D000202B0E9417130E94722B8091B50684FF19
:1062E0000AC082E891E00E94202B0E947F2843E0B0
:1062F00062E00E942F2B8EE791E00E94202B68968F
:106300000FB6F894DEBF0FBECDBFDF91CF911F91C6
:106310000F91FF90EF90DF90CF90BF90089587B1DD
:10632000887F87B988B1876088B9ECE6F0E0808122
:1063300087608083E8E6F0E0808182608083089552
:106340001F920F920FB60F9211242F933F934F93EA
:106350005F936F937F938F939F93AF93BF93EF93CD
:10636000FF9386B18095877099F080FF03C00E94EB
:10637000BC080EC0982F947021F080914405826073
:1063800005C081FF05C08091440588608093440565
:10639000FF91EF91BF91AF919F918F917F916F91FD
:1063A0005F914F913F912F910F900FBE0F901F90D3
:1063B000189580E008951F93CF93DF93EC0110E0D0
:1063C000BE01812F0E94FF20811102C087E009C019
:1063D0008881882341F0CE010E94142BCE010E94B7
:1063E000FF080E94AB2C1F5F123051F7DF91CF9155
:1063F0001F9108958F929F92AF92BF92CF92DF929A
:10640000EF92FF921F93CF93DF93CDB7DEB729971B
:106410000FB6F894DEBF0FBECDBF7C0181E0898747
:10642000F7018181833479F034F4882349F0843290
:1064300009F040C008C0873431F08835D9F503C071
:106440000E94562D1AC0F7019281911138C18334F0
:10645000B1F01CF4843231F010C0873461F088351B
:10646000F9F00BC080912805887111F088E028C1EF
:106470000E945A2D02C00E94B72F80E021C1809156
:106480002805823021F40E94BC0885E006C08111F5
:10649000EDCF82E08093280584E00E94232DEDCF8C
:1064A00080912805813049F783E00E94232D1092C6
:1064B0002805E3CF909128059230C0F6893459F130
:1064C0002CF4833251F0883489F08AC08E3409F478
:1064D0006AC0823509F440C083C082E08987F70131
:1064E00082818111ECC00E94262FC7CF8091BE0609
:1064F00084FFE3C084E0809328050E94AC0880916B
:1065000027058111BACF109228050E94D115C70125
:106510000E94DB31B2CF82E08987F701828181114D
:1065200007C0C7010E941C21C7010E948030A5CF6F
:106530008D3309F0C4C083E0F701E80FF11D9081AD
:10654000DF0113979C938F5F90819111F5CF89871D
:10655000C7010E94D81F91CFF7018281833509F0CE
:10656000AEC08381843509F0AAC084818D3309F0DF
:10657000A6C086818111A3C085E089878581843288
:1065800039F08A3239F0833209F099C082E003C0D1
:1065900081E001C08FEF0E94F51F88E00E94232D4B
:1065A0000E94BC086ACF82E08987F701828181114D
:1065B00013C010E0B701812F0E94FF20811104C099
:1065C00087E00E94AB2C04C0B701812F0E94663087
:1065D0001F5F123079F751CF911148CF11E001C000
:1065E00010E0AE014B5F5F4FBE01675F7F4FC70199
:1065F0000E947A27811102C082E062C0898521E071
:10660000280F2987F701E80FF11D80818D3309F0EC
:1066100056C0112321F1822F90E0E22FF0E0D70144
:10662000AE0FBF1F3C91E81BF90BEE0DFF1D308331
:106630002F5F3C913111F1CF2987C7010E94FF08DC
:1066400081113EC06D817E818F8198850E943E3987
:106650000E94A636862FB7010E94CF1F0ECFAE0133
:106660004F5F5F4FBE01675F7F4FC7010E947A2770
:10667000882311F28985F701E80FF11D80818111CE
:106680001EC0CD80DE80EF80F88420E030E04FE750
:1066900053E4C701B6010E943538181684F089808A
:1066A0009A80AB80BC80C701B6010E94A636862FB7
:1066B000B501A4010E94662103C085E001C083E00A
:1066C00029960FB6F894DEBF0FBECDBFDF91CF91F4
:1066D0001F91FF90EF90DF90CF90BF90AF909F9071
:1066E0008F900895CF93DF9324E0629FE0011124FF
:1066F0008C0F9D1FFC0160817181828193810E94BA
:10670000D436CF57D94F288139814A815B810E9485
:106710003936DF91CF910895FF920F931F93CF9356
:10672000DF938B01EC01F12C6F2DC8010E947233B5
:106730006993799389939993F39483E0F812F4CF52
:10674000DF91CF911F910F91FF90089508950895C3
:10675000089595B121E030E0082E01C0220F0A947F
:10676000EAF7662319F0922B95B90895209529230D
:1067700025B90895843029F021E0853019F020E012
:1067800001C022E09091CF06922321E009F420E09D
:1067900095B1621751F021E030E0082E01C0220FC0
:1067A0000A94EAF7922B95B9089521E030E0082E7B
:1067B00001C0220F0A94EAF72095292325B90895EC
:1067C00060E085E00E94BA3361E084E00C94BA3363
:1067D000009731F460E084E00E94BA3360E00CC0BE
:1067E0008130910511F40C94E033029741F460E09C
:1067F00084E00E94BA3361E085E00C94BA330895D6
:10680000249A259A87B1807387B982E090E00C942E
:10681000E8330C94003480E090E00C94E833CF939C
:10682000DF931F92CDB7DEB796B19073998329811C
:1068300030E0082E02C0359527950A94E2F72170C2
:106840003327843029F091E0853019F090E001C0C1
:1068500092E08091D006892319F481E0822701C05B
:10686000822F0F90DF91CF9108954F925F926F9298
:106870007F928F929F92AF92BF92CF92DF92EF92D0
:10688000FF920F931F93CF93DF938090D106909048
:10689000D206880C991C880C991CA12CB12C6091F3
:1068A000D3067091D4068091D5069091D6060E94A9
:1068B000A6362B01440C551C440C551CC1E0D0E0FD
:1068C000C12CD12C760111E001E0612C712C85E006
:1068D0000E940F3490E08C179D0771F5612F84E0C2
:1068E0000E94A933D501C4010197A109B10928F07B
:1068F0000000000000000000F7CF1027209739F7B4
:106900008FEFC81AD80AE80AF80A28ECC216D10490
:10691000E104F104E0F6C701B60124E130E040E013
:1069200050E00E946939672B682B692B81F6841827
:106930009508A608B708CBCF219748F6DF91CF91ED
:106940001F910F91FF90EF90DF90CF90BF90AF908D
:106950009F908F907F906F905F904F900895CF930E
:10696000C82F8C2F0E940F34882329F000000000CC
:1069700000000000F6CFCF910895CF93C82F8C2F41
:106980000E940F34811105C00000000000000000CB
:10699000F6CFCF91089580E090E00E94E8330E9406
:1069A000E03384E090E00E94BD3480E090E00E94FB
:1069B000E83382E090E00E94E83385E090E00C94B8
:1069C000BD340E94E03385E090E00E94AF3485E062
:1069D00090E00E94BD3480E090E00C94E83380E0C9
:1069E00094E39093D8068093D70686EA93E3909336
:1069F000DA068093D9068BEC94E39093DC068093BF
:106A0000DB068BE094E39093DE068093DD068091B5
:106A1000CE068130D9F08A30F9F489E094E390937E
:106A2000D8068093D70687EA93E39093DA0680939B
:106A3000D90685E394E39093DC068093DB0688EA2D
:106A400093E39093DE068093DD0606C081EE94E327
:106A50009093DC068093DB0687ED96E09093E0064A
:106A60008093DF06E091D706F091D80609948091D3
:106A700028058230E1F0E091DF06F091E006068023
:106A8000F781E02D09950E94A0150E94F3138091D3
:106A9000270581110CC0809128058111F6CFE09166
:106AA000DF06F091E0060480F581E02D0994089559
:106AB0005058BB27AA270ED076C23FD230F044D21E
:106AC00020F031F49F3F11F41EF40FC20EF4E09554
:106AD000E7FBDCC1E92F89D280F3BA17620773079D
:106AE0008407950718F071F49EF5B8C20EF4E0958E
:106AF0000B2EBA2FA02D0B01B90190010C01CA0178
:106B0000A0011124FF27591B99F0593F50F4503E22
:106B100068F11A16F040A22F232F342F4427585F14
:106B2000F3CF469537952795A795F0405395C9F72C
:106B30007EF41F16BA0B620B730B840BBAF09150E4
:106B4000A1F0FF0FBB1F661F771F881FC2F70EC083
:106B5000BA0F621F731F841F48F487957795679556
:106B6000B795F7959E3F08F0B3CF9395880F08F03F
:106B70009927EE0F979587950895DFD158F080E813
:106B800091E009F49EEFE0D128F040E851E059F49B
:106B90005EEF09C0AAC162C2E92FE07826D268F38D
:106BA000092E052AC1F3261737074807590738F079
:106BB0000E2E07F8E02569F0E025E0640AC0EF63D7
:106BC00007F8009407FADB01B9019D01DC01CA0155
:106BD000AD01EF935DD0E7D10AD05F91552331F03D
:106BE0002BED3FE049E450FD49EC63CF0895DF937E
:106BF000DD27B92FBF7740E85FE316161706480771
:106C00005B0710F4D92F35D29F938F937F936F93A7
:106C100032D3E2E3F1E06CD1C6D12F913F914F9195
:106C20005F916AD2DD2349F09058A2EA2AED3FE055
:106C300049EC5FE3D0785D274DDFDF91B4C1F7D138
:106C400080F09F3740F491110EF409C260E070E0CB
:106C500080E89FE3089526F01B16611D711D811DBC
:106C60001BC135C1EFD008F481E0089575D1E395DB
:106C7000ABC10CD098C168D140F05FD130F021F4A5
:106C80005F3F19F003C15111EAC12FC1AED198F392
:106C90009923C9F35523B1F3951B550BBB27AA279D
:106CA00062177307840738F09F5F5F4F220F331F0F
:106CB000441FAA1FA9F333D00E2E3AF0E0E830D0DB
:106CC00091505040E695001CCAF729D0FE2F27D0DE
:106CD000660F771F881FBB1F261737074807AB07AC
:106CE000B0E809F0BB0B802DBF01FF2793585F4F21
:106CF0002AF09E3F510568F0C9C0B1C15F3FECF377
:106D0000983EDCF3869577956795B795F7959F5FE5
:106D1000C9F7880F911D9695879597F90895E1E039
:106D2000660F771F881FBB1F621773078407BA0798
:106D300020F0621B730B840BBA0BEE1F88F7E095F3
:106D4000089504D06894B1118AC1089556D188F08D
:106D50009F5790F0B92F9927B751A0F0D1F0660F47
:106D6000771F881F991F1AF0BA95C9F712C0B13062
:106D700081F074D1B1E0089571C1672F782F882711
:106D8000B85F39F0B93FCCF3869577956795B395A1
:106D9000D9F73EF490958095709561957F4F8F4F10
:106DA0009F4F0895E89409C097FB3EF49095809515
:106DB000709561957F4F8F4F9F4F9923A9F0F92FC1
:106DC00096E9BB279395F695879577956795B7953F
:106DD000F111F8CFFAF4BB0F11F460FF1BC06F5F25
:106DE0007F4F8F4F9F4F16C0882311F096E911C037
:106DF000772321F09EE8872F762F05C0662371F058
:106E000096E8862F70E060E02AF09A95660F771F6B
:106E1000881FDAF7880F9695879597F9089507D117
:106E200080F09F3740F491110EF019C160E070E0DE
:106E300080E89FEB089526F41B16611D711D811DCE
:106E40002BC045C0990F0008550FAA0BE0E8FEEFD4
:106E500016161706E807F907C0F012161306E4071E
:106E6000F50798F0621B730B840B950B39F40A2617
:106E700061F0232B242B252B21F408950A2609F4F5
:106E8000A140A6958FEF811D811D089597F99F67F9
:106E900080E870E060E00895882371F4772321F0A2
:106EA0009850872B762F07C0662311F499270DC0C1
:106EB0009051862B70E060E02AF09A95660F771F5C
:106EC000881FDAF7880F9695879597F908959F3F61
:106ED00031F0915020F4879577956795B795880F95
:106EE000911D9695879597F908959FEF80EC0895E9
:106EF000DF93CF931F930F93FF92EF92DF927B016B
:106F00008C01689405C0DA2EEF01F6D0FE01E894FA
:106F1000A5912591359145915591AEF3EF01DADDBB
:106F2000FE019701A801DA9479F7DF90EF90FF90C6
:106F30000F911F91CF91DF91089500240A941616A6
:106F4000170618060906089500240A941216130657
:106F5000140605060895C9CF50D0E8F3E894E0E0A0
:106F6000BB279F57F0F02AED3FE049EC06C0EE0F3B
:106F7000BB0F661F771F881F28F0B23A620773079E
:106F8000840728F0B25A620B730B840BE3959A9531
:106F900072F7803830F49A95BB0F661F771F881FF1
:106FA000D2F7904896CF092E0394000C11F4882351
:106FB00052F0BB0F40F4BF2B11F460FF04C06F5FB1
:106FC0007F4F8F4F9F4F0895EF93E0FF06C0A2EAD7
:106FD0002AED3FE049EC5FEB7DDDE5DF0F900394A8
:106FE00001FC9058EFE5F1E057C157FD9058440F70
:106FF000551F59F05F3F71F04795880F97FB991F18
:1070000061F09F3F79F087950895121613061406D4
:10701000551FF2CF4695F1DF08C016161706180661
:10702000991FF1CF86957105610508940895E5DFF4
:10703000A0F0BEE7B91788F4BB279F3860F4161696
:10704000B11D672F782F8827985FF7CF86957795A2
:107050006795B11D93959639C8F30895E894BB27B9
:1070600066277727CB0197F90895ECDE08F48FEFB8
:1070700008959B01AC0160E070E080E89FE3F9CDEA
:10708000BCDF58F19E5758F19851A0F0E9F09830C4
:1070900020F5092E9927660F771F881F991F0A94DC
:1070A000D1F712C0062E672F782F8827985F11F42A
:1070B000000C07C0993FB4F3869577956795939533
:1070C000D9F7611D711D811D3EF4909580957095D5
:1070D00061957F4F8F4F9F4F08956894C0CFBECF6B
:1070E0000BD061CF2ADF28F02FDF18F0952309F0AD
:1070F000CDCEFBCE1124B3CF78DFA0F3959FD1F393
:10710000950F50E0551F629FF001729FBB27F00D55
:10711000B11D639FAA27F00DB11DAA1F649F6627AA
:10712000B00DA11D661F829F2227B00DA11D621FF9
:10713000739FB00DA11D621F839FA00D611D221FB3
:10714000749F3327A00D611D231F849F600D211D97
:10715000822F762F6A2F11249F5750408AF0E1F03A
:1071600088234AF0EE0FFF1FBB1F661F771F881F83
:1071700091505040A9F79E3F510570F087CE6FCFD8
:107180005F3FECF3983EDCF3869577956795B7956E
:10719000F795E7959F5FC1F7FE2B880F911D969598
:1071A000879597F9089529DFE0F09E37D8F0963952
:1071B000B8F49E3848F4672F782F8827985FF9CF66
:1071C00086957795679593959539D0F3B62FB170DD
:1071D0006B0F711D811D20F48795779567959395A9
:1071E0005BCE75CE3CCF9F93B7DE0F9007FCEE5F72
:1071F000EBCE11F40EF479CE6ACEFFDED0F39923F4
:10720000D9F3CEF39F57550B87FF3FD00024A0E65C
:1072100040EA900180585695979528F4805C660F57
:10722000771F881F20F026173707480730F4621BA6
:10723000730B840B202931294A2BA69517940794A8
:10724000202531254A2758F7660F771F881F20F021
:1072500026173707480730F4620B730B840B200D99
:10726000311D411DA09581F7B901842F9158880FD8
:107270009695879508959B01AC0132CFD8DE20F01A
:107280009F3708F4ECCE08CE22CE91505040660FC6
:10729000771F881FD2F708959F938F937F936F93E3
:1072A000FF93EF939B01AC011BDFEF91FF9120DE79
:1072B0002F913F914F915F9113CF991B79E004C0BB
:1072C000991F961708F0961B881F7A95C9F7809525
:1072D0000895A1E21A2EAA1BBB1BFD010DC0AA1F17
:1072E000BB1FEE1FFF1FA217B307E407F50720F02F
:1072F000A21BB30BE40BF50B661F771F881F991FAA
:107300001A9469F760957095809590959B01AC01F2
:10731000BD01CF010895EE0FFF1F0590F491E02D00
:1073200009940E949C39A59F900DB49F900DA49F35
:10733000800D911D11240895A29FB001B39FC0013B
:10734000A39F700D811D1124911DB29F700D811D91
:0A7350001124911D0895F894FFCF59
:00000001FF
